:020000040000FA
:0400000042EF35F0A6
:0400080003EF2FF0E3
:04001800B8EF21F02C
:06002A00D9CFE5FFE1CF94
:10003000D9FF00C0E5FF01C0E5FF02C0E5FF03C036
:10004000E5FF04C0E5FF05C0E5FF0001CF51D8B4CE
:100050002EEF00F00001CF6B30EF00F04CEF0BF013
:1000600060C300F00050210A02E181EF01F000506E
:10007000240A02E11EEF0AF000502A0A02E142EFD0
:1000800004F000502B0A02E163EF04F000502D0A47
:1000900002E1C8EF04F000503F0A02E1D9EF00F09E
:1000A0000050410A02E165EF08F00050420A02E107
:1000B00084EF09F00050430A02E1B1EF01F0005073
:1000C000440A02E1D7EF05F00050450A02E11FEFB4
:1000D00007F00050460A02E126EF09F00050490AF5
:1000E00002E15DEF0AF000504B0A02E1DBEF01F0A4
:1000F00000504C0A02E1B9EF02F000504E0A02E152
:100100007CEF06F00050500A02E1C2EF07F0005009
:10011000520A02E1D2EF0AF00050530A02E19EEFC8
:100120000AF00050540A02E12DEF05F00050580A81
:1001300002E114EF04F000505A0A02E1CAEF08F09D
:1001400000505E0A02E11CEF01F00050620A02E179
:10015000F1EF09F00050640A02E150EF06F00050A0
:10016000650A02E196EF07F00050660A02E157EFD8
:1001700009F000506C0A02E19CEF03F000506E0A97
:1001800002E1F3EF06F00050700A02E139EF08F0E7
:100190000050730A02E106EF0BF00050740A02E10E
:1001A000AAEF05F00050780A02E155EF04F030EFB5
:1001B0000BF0E60EF66E1D0EF76E000EF86E0900DF
:1001C000F5CF00F00900F5CF01F00900F5CF02F0FE
:1001D0000250E56E0150E56E0050E56E45EC31F0E1
:1001E000030EE1260001D351E56E0001D251E56E08
:1001F0000001D151E56E0001D051E56E000EE56EB3
:100200001E0EE56E620EE56E000EE56E1E0EE56ECC
:100210005C0EE56E03010151E56E03010051E56ED0
:10022000000EE56E1E0EE56E140EE56E45EC31F027
:100230000F0EE1264CEF0BF003016251300A02E190
:100240002AEF01F003016251310A02E12AEF01F0C5
:1002500059EF01F0D00E03016225006E005003013A
:10026000306F60C300F0016A0001D351E56E0001F8
:10027000D251E56E0001D151E56E0001D051E56E1D
:100280000150E56E0050E56E03010151E56E03017A
:100290000051E56E0001CB51E56E0001CA51E56EDB
:1002A0000001C951E56E45EC31F00B0EE1264CEF33
:1002B0000BF060C300F0016A0001D351E56E00014C
:1002C000D251E56E0001D151E56E0001D051E56ECD
:1002D0000150E56E0050E56E03010151E56E03012A
:1002E0000051E56E0001CE51E56E0001CD51E56E85
:1002F0000001CC51E56E45EC31F00B0EE1264CEFE0
:100300000BF0100EE56E21EC34F0E12A60C300F032
:10031000016A0001D351E56E0001D251E56E000182
:10032000D151E56E0001D051E56E0150E56E0050EF
:10033000E56E03010151E56E03010051E56E000118
:10034000CB51E56E0001CA51E56E0001C951E56E61
:1003500045EC31F00B0EE126010E0001686F4CEF09
:100360000BF060C300F0016A0001D351E56E00019B
:10037000D251E56E0001D151E56E0001D051E56E1C
:100380000150E56E0050E56E03010151E56E030179
:100390000051E56E0001CB51E56E0001CA51E56EDA
:1003A0000001C951E56E45EC31F00B0EE126EFEC92
:1003B00014F04CEF0BF0300E0301625DD8A0E7EFB4
:1003C00001F0380E0301625DD8A00FEF02F060C3A8
:1003D00000F0016A0001D351E56E0001D251E56ED3
:1003E0000001D151E56E0001D051E56E0150E56E7E
:1003F0000050E56E03010151E56E03010051E56E09
:100400000001CE51E56E0001CD51E56E0001CC51E9
:10041000E56E45EC31F00B0EE1264CEF0BF064C3BA
:1004200000F00050300A02E11DEF02F00050310AE6
:1004300002E157EF02F091EF02F0D00E03016225C6
:10044000006E010E016E005005E0E86CD890013698
:10045000010FFDE30150E56EA7EC33F0E12A60C324
:1004600000F0016A0001D351E56E0001D251E56E42
:100470000001D151E56E0001D051E56E0150E56EED
:100480000050E56E03010151E56E03010051E56E78
:100490000001CB51E56E0001CA51E56E0001C95162
:1004A000E56E45EC31F00B0EE1264CEF0BF0D00E73
:1004B00003016225006E010E016E005005E0E86C3C
:1004C000D8900136010FFDE30150E56EB8EC34F031
:1004D000E12A60C300F0016A0001D351E56E00011A
:1004E000D251E56E0001D151E56E0001D051E56EAB
:1004F0000150E56E0050E56E03010151E56E030108
:100500000051E56E0001CB51E56E0001CA51E56E68
:100510000001C951E56E45EC31F00B0EE1264CEFC0
:100520000BF060C300F0016A0001D351E56E0001D9
:10053000D251E56E0001D151E56E0001D051E56E5A
:100540000150E56E0050E56E03010151E56E0301B7
:100550000051E56E0001CE51E56E0001CD51E56E12
:100560000001CC51E56E45EC31F00B0EE1264CEF6D
:100570000BF0300E0301625DD8A0CAEF02F0380E16
:100580000301625DD8B0CAEF02F003010251D8A4A2
:10059000F2EF02F060C300F0016A0001D351E56E92
:1005A0000001D251E56E0001D151E56E0001D0513C
:1005B000E56E0150E56E0050E56E03010151E56EF8
:1005C00003010051E56E0001CE51E56E0001CD51F1
:1005D000E56E0001CC51E56E45EC31F00B0EE126E5
:1005E0004CEF0BF064C300F00050300A02E100EF62
:1005F00003F00050310A02E13AEF03F074EF03F028
:10060000D00E03016225006E010E016E005005E060
:10061000E86CD8900136010FFDE30150E56EC6ECA1
:1006200033F0E12A60C300F0016A0001D351E56EA6
:100630000001D251E56E0001D151E56E0001D051AB
:10064000E56E0150E56E0050E56E03010151E56E67
:1006500003010051E56E0001CB51E56E0001CA5166
:10066000E56E0001C951E56E45EC31F00B0EE12657
:100670004CEF0BF0D00E03016225006E010E016EEF
:10068000005005E0E86CD8900136010FFDE3015001
:10069000E56E21EC34F0E12A60C300F0016A00014C
:1006A000D351E56E0001D251E56E0001D151E56EE6
:1006B0000001D051E56E0150E56E0050E56E03017A
:1006C0000151E56E03010051E56E0001CB51E56E6D
:1006D0000001CA51E56E0001C951E56E45EC31F0EB
:1006E0000B0EE1264CEF0BF060C300F0016A000135
:1006F000D351E56E0001D251E56E0001D151E56E96
:100700000001D051E56E0150E56E0050E56E030129
:100710000151E56E03010051E56E0001CE51E56E19
:100720000001CD51E56E0001CC51E56E45EC31F094
:100730000B0EE1264CEF0BF0300E0301625DD8A0EA
:10074000ECEF03F0380E0301625DD8B0ECEF03F07C
:1007500002C300F0016AD00E03016225026E010E91
:10076000036E025005E0E86CD8900336010FFDE3FC
:100770000350E56E1AEC33F0026EE12A036A60C39F
:1007800004F0056A0001D351E56E0001D251E56E17
:100790000001D151E56E0001D051E56E0150E56ECA
:1007A0000050E56E0350E56E0250E56E0550E56EB3
:1007B0000450E56E03010151E56E03010051E56E41
:1007C000000EE56E1E0EE56E700EE56E45EC31F026
:1007D0000F0EE1264CEF0BF060C300F0016A000140
:1007E000D351E56E0001D251E56E0001D151E56EA5
:1007F0000001D051E56E0150E56E0050E56E030139
:100800000151E56E03010051E56E0001CE51E56E28
:100810000001CD51E56E0001CC51E56E45EC31F0A3
:100820000B0EE1264CEF0BF003016251E56EE0EC9C
:1008300034F0E12A60C300F0016A0001D351E56E93
:100840000001D251E56E0001D151E56E0001D05199
:10085000E56E0150E56E0050E56E03010151E56E55
:1008600003010051E56E0001CB51E56E0001CA5154
:10087000E56E0001C951E56E45EC31F00B0EE12645
:100880004CEF0BF0010EE56E7BEC22F0E12A61ECFF
:1008900035F0006E03016051E56E0050E56EEBEC43
:1008A00023F0020EE1264CEF0BF061EC35F0006E08
:1008B00003016051E56E0050E56EEBEC23F0020E93
:1008C000E1264CEF0BF0300E0301625DD8A0A0EFE3
:1008D00004F0380E0301625DD8B0A0EF04F0D00E32
:1008E00003016225006E0050E56E65EC33F0E12AED
:1008F00060C300F0016A0001D351E56E0001D251DE
:10090000E56E0001D151E56E0001D051E56E015058
:10091000E56E0050E56E03010151E56E03010051E3
:10092000E56E0001CB51E56E0001CA51E56E000194
:10093000C951E56E45EC31F00B0EE1264CEF0BF0A2
:1009400060C300F0016A0001D351E56E0001D2518D
:10095000E56E0001D151E56E0001D051E56E015008
:10096000E56E0050E56E03010151E56E0301005193
:10097000E56E0001CE51E56E0001CD51E56E00013E
:10098000CC51E56E45EC31F00B0EE1264CEF0BF04F
:10099000300E0301625DD8A005EF05F0380E0301AB
:1009A000625DD8B005EF05F0D00E03016225006E40
:1009B0000050E56E42EC33F0E12A60C300F0016ABA
:1009C0000001D351E56E0001D251E56E0001D15115
:1009D000E56E0001D051E56E0150E56E0050E56E08
:1009E00003010151E56E03010051E56E0001CB5199
:1009F000E56E0001CA51E56E0001C951E56E45EC96
:100A000031F00B0EE1264CEF0BF060C300F0016AF1
:100A10000001D351E56E0001D251E56E0001D151C4
:100A2000E56E0001D051E56E0150E56E0050E56EB7
:100A300003010151E56E03010051E56E0001CE5145
:100A4000E56E0001CD51E56E0001CC51E56E45EC3F
:100A500031F00B0EE1264CEF0BF0030E016E620E2F
:100A6000006E800E026E0250E56E0150E56E005081
:100A7000E56EF0EC20F0006EF3CF01F0030EE126FE
:100A800000500301A36F2C0E0301A35DD8B082EFC9
:100A900005F0020E0301A35DD8A082EF05F0A3C309
:100AA00000F0016A0150E56E0050E56E82EC30F016
:100AB000020EE12660C300F0016A0001D351E56E29
:100AC0000001D251E56E0001D151E56E0001D05117
:100AD000E56E0150E56E0050E56E03010151E56ED3
:100AE00003010051E56E0001CB51E56E0001CA51D2
:100AF000E56E0001C951E56E45EC31F00B0EE126C3
:100B00004CEF0BF060C300F0016A0001D351E56EB9
:100B10000001D251E56E0001D151E56E0001D051C6
:100B2000E56E0150E56E0050E56E03010151E56E82
:100B300003010051E56E0001CE51E56E0001CD517B
:100B4000E56E0001CC51E56E45EC31F00B0EE1266F
:100B50004CEF0BF058EC35F0006E016A60C302F008
:100B6000036A0001D351E56E0001D251E56E000128
:100B7000D151E56E0001D051E56E0150E56E005097
:100B8000E56E0350E56E0250E56E03010151E56E1E
:100B900003010051E56E000EE56E1E0EE56E940E2B
:100BA000E56E45EC31F00D0EE1264CEF0BF0030E37
:100BB000016E620E006E800E026E0250E56E0150F4
:100BC000E56E0050E56EF0EC20F0006EF3CF01F022
:100BD000030EE12600500301A36F0301A351D8B413
:100BE000FAEF05F00301A351010A02E1FAEF05F063
:100BF00028EF06F00301A351E56EC1EC31F0E12AC4
:100C000060C300F0016A0001D351E56E0001D251CA
:100C1000E56E0001D151E56E0001D051E56E015045
:100C2000E56E0050E56E03010151E56E03010051D0
:100C3000E56E0001CB51E56E0001CA51E56E000181
:100C4000C951E56E45EC31F00B0EE1264CEF0BF08F
:100C500060C300F0016A0001D351E56E0001D2517A
:100C6000E56E0001D151E56E0001D051E56E0150F5
:100C7000E56E0050E56E03010151E56E0301005180
:100C8000E56E0001CE51E56E0001CD51E56E00012B
:100C9000CC51E56E45EC31F00B0EE1264CEF0BF03C
:100CA0002CC300F0016A60C302F0036A0001D35153
:100CB000E56E0001D251E56E0001D151E56E0001F3
:100CC000D051E56E0150E56E0050E56E0350E56EC3
:100CD0000250E56E03010151E56E03010051E56E1E
:100CE000000EE56E1E0EE56E940EE56E45EC31F0DD
:100CF0000D0EE1264CEF0BF0030E016E620E006E3E
:100D0000800E026E0250E56E0150E56E0050E56EF9
:100D1000F0EC20F0006EF3CF01F0030EE12600505E
:100D20000301A36F0301A351D8B49FEF06F00301A1
:100D3000A351010A02E19FEF06F0CBEF06F0030199
:100D4000A35103012D6F60C300F0016A0001D3516C
:100D5000E56E0001D251E56E0001D151E56E000152
:100D6000D051E56E0150E56E0050E56E0301015172
:100D7000E56E03010051E56E0001CB51E56E000107
:100D8000CA51E56E0001C951E56E45EC31F00B0E1C
:100D9000E1264CEF0BF060C300F0016A0001D35173
:100DA000E56E0001D251E56E0001D151E56E000102
:100DB000D051E56E0150E56E0050E56E0301015122
:100DC000E56E03010051E56E0001CE51E56E0001B4
:100DD000CD51E56E0001CC51E56E45EC31F00B0EC6
:100DE000E1264CEF0BF02DC300F0016A60C302F066
:100DF000036A0001D351E56E0001D251E56E000196
:100E0000D151E56E0001D051E56E0150E56E005004
:100E1000E56E0350E56E0250E56E03010151E56E8B
:100E200003010051E56E000EE56E1E0EE56E940E98
:100E3000E56E45EC31F00D0EE1264CEF0BF0030EA4
:100E4000016E620E006E800E026E0250E56E015061
:100E5000E56E0050E56EF0EC20F0006EF3CF01F08F
:100E6000030EE12600500301A36F0301A351D8B480
:100E700042EF07F00301A351010A02E142EF07F03C
:100E80006EEF07F00301A35103012F6F60C300F061
:100E9000016A0001D351E56E0001D251E56E0001F7
:100EA000D151E56E0001D051E56E0150E56E005064
:100EB000E56E03010151E56E03010051E56E00018D
:100EC000CB51E56E0001CA51E56E0001C951E56ED6
:100ED00045EC31F00B0EE1264CEF0BF060C300F057
:100EE000016A0001D351E56E0001D251E56E0001A7
:100EF000D151E56E0001D051E56E0150E56E005014
:100F0000E56E03010151E56E03010051E56E00013C
:100F1000CE51E56E0001CD51E56E0001CC51E56E7C
:100F200045EC31F00B0EE1264CEF0BF02FC300F037
:100F3000016A60C302F0036A0001D351E56E00014B
:100F4000D251E56E0001D151E56E0001D051E56E40
:100F50000150E56E0050E56E0350E56E0250E56EFF
:100F600003010151E56E03010051E56E000EE56ECF
:100F70001E0EE56E940EE56E45EC31F00D0EE12689
:100F80004CEF0BF0030E016E620E006E800E026ECF
:100F90000250E56E0150E56E0050E56EF0EC20F079
:100FA000006EF3CF01F0030EE12600500301A36FA2
:100FB0000301A351D8B4E5EF07F00301A351010ADF
:100FC00002E1E5EF07F011EF08F00301A35103017F
:100FD0002E6F60C300F0016A0001D351E56E00017D
:100FE000D251E56E0001D151E56E0001D051E56EA0
:100FF0000150E56E0050E56E03010151E56E0301FD
:101000000051E56E0001CB51E56E0001CA51E56E5D
:101010000001C951E56E45EC31F00B0EE1264CEFB5
:101020000BF060C300F0016A0001D351E56E0001CE
:10103000D251E56E0001D151E56E0001D051E56E4F
:101040000150E56E0050E56E03010151E56E0301AC
:101050000051E56E0001CE51E56E0001CD51E56E07
:101060000001CC51E56E45EC31F00B0EE1264CEF62
:101070000BF02EC300F0016A60C302F0036A0001A6
:10108000D351E56E0001D251E56E0001D151E56EFC
:101090000001D051E56E0150E56E0050E56E035041
:1010A000E56E0250E56E03010151E56E030100514A
:1010B000E56E000EE56E1E0EE56E940EE56E45ECD7
:1010C00031F00D0EE1264CEF0BF003012B51D8A4AB
:1010D000A2EF08F0100EE56E21EC34F0E12A010ECB
:1010E00003012B6F0001D06B0001D16B0001D26BAB
:1010F0000001D36B60C300F0016A0001D351E56EBB
:101100000001D251E56E0001D151E56E0001D051D0
:10111000E56E0150E56E0050E56E03010151E56E8C
:1011200003010051E56E0001CB51E56E0001CA518B
:10113000E56E0001C951E56E45EC31F00B0EE1267C
:101140004CEF0BF060C300F0016A0001D351E56E73
:101150000001D251E56E0001D151E56E0001D05180
:10116000E56E0150E56E0050E56E03010151E56E3C
:1011700003010051E56E0001CE51E56E0001CD5135
:10118000E56E0001CC51E56E45EC31F00B0EE12629
:101190004CEF0BF003012B51D8B4FEEF08F0100E0A
:1011A000E56EC6EC33F0E12A03012B6B60C300F05F
:1011B000016A0001D351E56E0001D251E56E0001D4
:1011C000D151E56E0001D051E56E0150E56E005041
:1011D000E56E03010151E56E03010051E56E00016A
:1011E000CB51E56E0001CA51E56E0001C951E56EB3
:1011F00045EC31F00B0EE1264CEF0BF060C300F034
:10120000016A0001D351E56E0001D251E56E000183
:10121000D151E56E0001D051E56E0150E56E0050F0
:10122000E56E03010151E56E03010051E56E000119
:10123000CE51E56E0001CD51E56E0001CC51E56E59
:1012400045EC31F00B0EE1264CEF0BF0D00E030114
:101250006225006E0050E56E02EC35F0E12A60C3B5
:1012600000F0016A0001D351E56E0001D251E56E34
:101270000001D151E56E0001D051E56E0150E56EDF
:101280000050E56E03010151E56E03010051E56E6A
:101290000001CB51E56E0001CA51E56E0001C95154
:1012A000E56E45EC31F00B0EE1264CEF0BF073ECE4
:1012B00035F0006E016A60C302F0036A0001D35189
:1012C000E56E0001D251E56E0001D151E56E0001DD
:1012D000D051E56E0150E56E0050E56E0350E56EAD
:1012E0000250E56E03010151E56E03010051E56E08
:1012F000000EE56E1E0EE56E940EE56E45EC31F0C7
:101300000D0EE1264CEF0BF0030E016E620E006E27
:10131000800E026E0250E56E0150E56E0050E56EE3
:10132000F0EC20F0006EF3CF01F0030EE126005048
:10133000E56E68EC32F0006EE12A0050D8B4C9EFD7
:1013400009F060C300F0016A0001D351E56E0001AD
:10135000D251E56E0001D151E56E0001D051E56E2C
:101360000150E56E0050E56E03010151E56E030189
:101370000051E56E0001CB51E56E0001CA51E56EEA
:101380000001C951E56E45EC31F00B0EE1264CEF42
:101390000BF060C300F0016A0001D351E56E00015B
:1013A000D251E56E0001D151E56E0001D051E56EDC
:1013B0000150E56E0050E56E03010151E56E030139
:1013C0000051E56E0001CE51E56E0001CD51E56E94
:1013D0000001CC51E56E45EC31F00B0EE1264CEFEF
:1013E0000BF06AEC35F0006E016A60C302F0036A2C
:1013F0000001D351E56E0001D251E56E0001D151DB
:10140000E56E0001D051E56E0150E56E0050E56ECD
:101410000350E56E0250E56E03010151E56E0301D4
:101420000051E56E000EE56E1E0EE56E940EE56E43
:1014300045EC31F00D0EE1264CEF0BF0300E0301C0
:10144000625DD8A035EF0AF0380E0301625DD8B0B6
:1014500035EF0AF0D00E03016225006E0050E56EF4
:101460004EEC25F0E12A4CEF0BF060C300F0016A6E
:101470000001D351E56E0001D251E56E0001D1515A
:10148000E56E0001D051E56E0150E56E0050E56E4D
:1014900003010151E56E03010051E56E0001CE51DB
:1014A000E56E0001CD51E56E0001CC51E56E45ECD5
:1014B00031F00B0EE1264CEF0BF0030E016E620EC5
:1014C000006E800E026E0250E56E0150E56E005017
:1014D000E56EF0EC20F0006EF3CF01F0030EE12694
:1014E00000500301006F01500301016F60C300F061
:1014F000016A0001D351E56E0001D251E56E000191
:10150000D151E56E0001D051E56E0150E56E0050FD
:10151000E56E03010151E56E03010051E56E000126
:10152000CB51E56E0001CA51E56E0001C951E56E6F
:1015300045EC31F00B0EE1264CEF0BF0100EE56E92
:1015400021EC34F0E12A3DEC27F0100EE56EC6ECFC
:1015500033F0E12A60C300F0016A0001D351E56E67
:101560000001D251E56E0001D151E56E0001D0516C
:10157000E56E0150E56E0050E56E03010151E56E28
:1015800003010051E56E0001CB51E56E0001CA5127
:10159000E56E0001C951E56E45EC31F00B0EE12618
:1015A0004CEF0BF0100EE56E21EC34F0E12A7BECF1
:1015B0002DF0100EE56EC6EC33F0E12A60C300F0AA
:1015C000016A0001D351E56E0001D251E56E0001C0
:1015D000D151E56E0001D051E56E0150E56E00502D
:1015E000E56E03010151E56E03010051E56E000156
:1015F000CB51E56E0001CA51E56E0001C951E56E9F
:1016000045EC31F00B0EE1264CEF0BF014EC2DF015
:1016100060C300F0016A0001D351E56E0001D251B0
:10162000E56E0001D151E56E0001D051E56E01502B
:10163000E56E0050E56E03010151E56E03010051B6
:10164000E56E0001CB51E56E0001CA51E56E000167
:10165000C951E56E45EC31F00B0EE1264CEF0BF075
:101660000001D351E56E0001D251E56E0001D15168
:10167000E56E0001D051E56E03010151E56E0301F5
:101680000051E56E000EE56E1E0EE56EA80EE56ECD
:1016900045EC31F0090EE126E4CF05F0E4CF04F08B
:1016A000E4CF03F0E4CF02F0E4CF01F0E4CF00F0A8
:1016B000E4CFD9FF1200D9CFE5FFE1CFD9FF00C0B9
:1016C000E5FF01C0E5FF02C0E5FF03C0E5FF04C080
:1016D000E5FF05C0E5FF06C0E5FF07C0E5FF08C060
:1016E000E5FF09C0E5FF0AC0E5FF0BC0E5FF0CC040
:1016F000E5FF0DC0E5FF0EC0E5FF0FC0E5FF10C020
:10170000E5FF11C0E5FF12C0E5FF13C0E5FF14C0FF
:10171000E5FF15C0E5FF16C0E5FF17C0E5FF18C0DF
:10172000E5FF020EDBCF00F0D8900034016E810E91
:101730000124026E036A000E0322710E0124046E5E
:10174000056A000E052204C0E9FF05C0EAFFEECFDE
:1017500004F0EFCF05F00050200DF3CF06F0F4CFEA
:1017600007F0000E0624086E010E0720096E6AC0FD
:101770000AF00B6A29C30CF00D6A0C500A260D50B2
:101780000B22FF0E0A26D8A00B0629C30CF00D6A07
:101790000D50E56E0C50E56E0B50E56E0A50E56E8F
:1017A00039EC2CF00A6EF3CF0BF0040EE1260B504F
:1017B000E56E0A50E56E000EE56E020EE56EABECCE
:1017C0002FF00A6EF3CF0BF0040EE1260A50082624
:1017D0000B50092208C0E9FF09C0EAFFEECF08F06C
:1017E000EFCF09F00950E56E0850E56E0550E56E43
:1017F0000450E56EFBEC2FF0046EF3CF05F0040E01
:10180000E12602C0E9FF03C0EAFF04C0EEFF05C005
:10181000EFFF710E0124026E036A000E03220050D6
:10182000E56E56EC19F0046EF3CF05F0E12A02C024
:10183000E9FF03C0EAFF04C0EEFF05C0EFFF0301AC
:101840003051D8B4A3EF0CF06CC002F0036A150E4F
:101850000124046E056A030E052204C0E9FF05C0D9
:10186000EAFFEECF04F0EFCF05F0086A096A810EB7
:1018700001240A6E0B6A000E0B220AC0E9FF0BC09E
:10188000EAFFEECF0AF0EFCF0BF00C6A0D6A710E93
:1018900001240E6E0F6A000E0F220EC0E9FF0FC06A
:1018A000EAFFEECF0EF0EFCF0FF0106A116A000ED4
:1018B0000626010E072200016A05126ED890123624
:1018C00012500626E86A072206C0E9FF07C0EAFFB1
:1018D000EECF06F0EFCF07F0126A136A00C014F0E3
:1018E000156A0350E56E0250E56E0950E56E08502A
:1018F000E56E0550E56E0450E56E0D50E56E0C503A
:10190000E56E0B50E56E0A50E56E1150E56E105015
:10191000E56E0F50E56E0E50E56E1350E56E1250F9
:10192000E56E0750E56E0650E56E1550E56E1450F5
:10193000E56E000EE56E350EE56E520EE56E45EC79
:1019400031F0170EE126710E0124026E036A000EBB
:10195000032202C0E9FF03C0EAFFEECF02F0EFCF9F
:1019600003F0810E0124046E056A000E052204C0F6
:10197000E9FF05C0EAFFEECF04F0EFCF05F0150E4A
:101980000124066E076A030E072206C0E9FF07C09E
:10199000EAFFEECF06F0EFCF07F00550075C02E15B
:1019A0000450065CD8A0FDEF0CF00050E56E56EC3C
:1019B00019F0026EF3CF03F0E12A03012905046E4A
:1019C0000450E56E45EC2EF0E12A03013051D8B405
:1019D00085EF0DF000C004F0056A0550E56E045077
:1019E000E56E000EE56E350EE56E9A0EE56E45EC81
:1019F00031F0050EE12685EF0DF0080E046E080E9D
:101A0000056E0550D8B485EF0DF0810E0124066EE9
:101A1000076A000E072206C0E9FF07C0EAFFEECF03
:101A200006F0EFCF07F0150E0124086E096A030EC9
:101A3000092208C0E9FF09C0EAFFEECF08F0EFCFA6
:101A400009F005C00AF00B6A0B50E56E0A50E56E0E
:101A50000950E56E0850E56EABEC2FF0086EF3CF41
:101A600009F0040EE1263FEC30F00A6E0B6A0B50D1
:101A7000E56E0A50E56E0950E56E0850E56EABEC78
:101A80002FF0086EF3CF09F0040EE1260750095C31
:101A900002E10650085CD8B080EF0DF00450080851
:101AA000066ED8900636062A0650E56E45EC2EF0F6
:101AB000E12A0050E56E56EC19F0026EF3CF03F008
:101AC000E12A03013051D8B485EF0DF004C006F0CF
:101AD000076A00C008F0096A0750E56E0650E56E17
:101AE0000950E56E0850E56E000EE56E350EE56EA8
:101AF000BE0EE56E45EC31F0070EE12685EF0DF0E8
:101B0000050605C004F001EF0DF003012C51D8B417
:101B1000A5EF0EF003013051D8B402EF0EF0C7C0AC
:101B200004F0C8C005F0066A076A810E0124086E39
:101B3000096A000E092208C0E9FF09C0EAFFEECFDA
:101B400008F0EFCF09F00A6A0B6AC5C00CF0C6C0F6
:101B50000DF00E6A0F6A050E0124106E116A030E55
:101B6000112210C0E9FF11C0EAFFEECF10F0EFCF55
:101B700011F0126A136A710E0124146E156A000EB8
:101B8000152214C0E9FF15C0EAFFEECF14F0EFCF25
:101B900015F0166A176A186A0750E56E0650E56E6A
:101BA0000550E56E0450E56E0B50E56E0A50E56E8B
:101BB0000950E56E0850E56E0F50E56E0E50E56E6B
:101BC0000D50E56E0C50E56E1350E56E1250E56E4B
:101BD0001150E56E1050E56E1750E56E1650E56E2B
:101BE0001550E56E1450E56E1850E56E0050E56E28
:101BF000000EE56E350EE56EEC0EE56E45EC31F04F
:101C0000190EE126710E0124006E046A000E0422F2
:101C100000C0E9FF04C0EAFFEECF00F0EFCF04F010
:101C200003012551005E03012651045A050E0124CB
:101C3000056E066A030E062205C0E9FF06C0EAFF2C
:101C4000EECF05F0EFCF06F00550005E0650045AC7
:101C50000450E56E0050E56E78EC1AF0006EF3CF9C
:101C600004F0020EE1260001C651045C03E100010C
:101C7000C551005CD8B077EF0EF0810E0124006EE4
:101C8000046A000E042200C0E9FF04C0EAFFEECFA0
:101C900000F0EFCF04F00001C851045C03E1000143
:101CA000C751005CD8B077EF0EF0050E0124006E2E
:101CB000046A030E0422710E0124056E066A000EEA
:101CC000062205C0E9FF06C0EAFFEECF05F0EFCF20
:101CD00006F003012551055E03012651065A00C096
:101CE000E9FF04C0EAFF05C0EEFF06C0EFFF0301F5
:101CF0002551025C006E030126510358046E050E47
:101D00000124056E066A030E062205C0E9FF06C01F
:101D1000EAFFEECF07F0EFCF08F00850045C02E1D5
:101D20000750005CD8B0A5EF0EF003012551025C0E
:101D3000006E030126510358046E05C0E9FF06C07A
:101D4000EAFF00C0EEFF04C0EFFF03012D51D8B43D
:101D5000BBEF0EF0006A050E0126030E002201C043
:101D6000E9FF00C0EAFFEECF01F0EFCF00F0015035
:101D7000025E0050035A03C0F3FF0250E4CF18F094
:101D8000E4CF17F0E4CF16F0E4CF15F0E4CF14F071
:101D9000E4CF13F0E4CF12F0E4CF11F0E4CF10F071
:101DA000E4CF0FF0E4CF0EF0E4CF0DF0E4CF0CF071
:101DB000E4CF0BF0E4CF0AF0E4CF09F0E4CF08F071
:101DC000E4CF07F0E4CF06F0E4CF05F0E4CF04F071
:101DD000E4CF03F0E4CF02F0E4CF01F0E4CF00F071
:101DE000E4CFD9FF1200D41E0000494E464F2C25E7
:101DF000642C25632C25732C256C640D0A00564138
:101E00004C55452C25642C25642C256C642C256CA4
:101E1000640D0A00494E464F2C25642C43617042E4
:101E20006F617264204669726D77617265202573F7
:101E3000202D204275696C643A2025732C687474D7
:101E4000703A2F2F7777772E63617073656E7365A5
:101E50002E6F72672C256C640D0A000076322E30CE
:101E6000000032303038313030365F3134323700B4
:101E7000494E464F2C25642C25632C25642028755B
:101E80007365204C4544533A202564292C256C6405
:101E90000D0A0000494E464F2C25642C25632C2545
:101EA000642C256C640D0A005245504C592C256455
:101EB0002C434F4D4D414E44204E4F5420524543EC
:101EC0004F474E495A45442C4552524F522C256C8F
:101ED000640D0A0053686F727420636F6D6D616EDC
:101EE000642068656C7020666F7220436170426F79
:101EF0006172642076322E303A0D0A28436F6D707D
:101F00006C65746520616C6C20636F6D6D616E64CF
:101F1000732077697468203C454E5445523E290D24
:101F20000A0D0A5B47656E6572616C5D0D0A4109B9
:101F300009097374617274206D6561737572696EDD
:101F4000670D0A5A09090973746F70206D65617312
:101F50007572696E670D0A2B2078090909656E6133
:101F6000626C65206368616E6E656C207820283035
:101F70002D37290D0A2D20780909096469736162DA
:101F80006C65206368616E6E656C20782028302D4A
:101F900037290D0A2A20200909096175746F2D64FB
:101FA000657465637420636F6E6E65637465642029
:101FB00073656E736F72730D0A43202009090961FE
:101FC00075746F2D64657465637420616E6420633D
:101FD000616C6962726174652073656E736F727390
:101FE0000D0A0D0A21202009090972657365742004
:101FF0006465766963650D0A3F20200909097072DE
:10200000696E7420746869732068656C70206D65F2
:1020100073736167650D0A5320200909097361769E
:102020006520636F6E66696775726174696F6E2093
:10203000746F20454550524F4D0D0A52202009091A
:1020400009726573746F726520636F6E6669677578
:10205000726174696F6E2066726F6D2045455052D3
:102060004F4D0D0A7320200909097072696E7420A2
:10207000454550524F4D20636F6E74656E747320EA
:102080006173206865780D0A0D0A5B46696C74659A
:1020900072696E675D0D0A462078090909736574D7
:1020A0002066696C746572206D6574686F642028A1
:1020B000783D20303A6E6F2066696C746572696E87
:1020C000672C20313A617665726167652C20323A5F
:1020D00061646170746976652061766572616765B7
:1020E000290D0A6620200909097072696E7420663C
:1020F000696C746572206D6574686F640D0A4420A4
:1021000078090909656E61626C652F6469736162A3
:102110006C6520647269667420636F6D70656E73A0
:102120006174696F6E2028783D312F30290D0A6463
:1021300020200909097072696E74207374617475C6
:1021400073206F6620647269667420636F6D7065BA
:102150006E736174696F6E0D0A5020780909096504
:102160006E61626C652F64697361626C6520617574
:10217000746F2D7265736574206F66207374756358
:102180006B206368616E6E656C732028783D312F1B
:1021900030290D0A7020200909097072696E7420B7
:1021A000737461747573206F66206175746F2D721E
:1021B000657365740D0A4E2078090909656E6162C0
:1021C0006C652F64697361626C652073656E736FF3
:1021D000722076616C7565206E6F726D616C697AC4
:1021E0006174696F6E2028783D312F30290D0A6E99
:1021F00020200909097072696E7420737461747506
:1022000073206F66206E6F726D616C697A6174699C
:102210006F6E0D0A42207809090973657420627592
:10222000666665722073697A652028783D312E2EA6
:102230003136290D0A6220200909097072696E740D
:10224000206275666665722073697A650D0A0D0AEB
:102250005B4C454473202F204750494F5D0D0A4C7D
:1022600020782079090909656E61626C652F6469BF
:102270007361626C65204C454420782028783D309D
:102280002E2E372C20793D312F30290D0A4B207806
:102290002079090909656E61626C652F6469736153
:1022A000626C6520626C696E6B696E67206F662078
:1022B0004C454420782028783D302E2E372C20792C
:1022C0003D312F30290D0A6C207820200909097032
:1022D00072696E7420737461747573206F66204C1C
:1022E0004544207820283D3E20303A6F66662C20F9
:1022F000313A6F6E2C20323A626C696E6B696E6790
:10230000290D0A0D0A5B416476616E6365645D0D9B
:102310000A5420780909097365742073616D706C23
:10232000696E672074696D652070657220636861ED
:102330006E6E656C20696E206D73202831302E2EF4
:102340003432290D0A7420200909097072696E74EB
:102350002073616D706C696E672074696D652070A3
:102360006572206368616E6E656C0D0A582078098D
:102370000909736574206163746976652063686117
:102380006E6E656C73202878206973206120382078
:10239000626974206269746D61736B290D0A78201B
:1023A000200909097072696E742061637469766529
:1023B000206368616E6E656C730D0A4920780909A7
:1023C0000973657420646576696365204944202833
:1023D000783D302E2E363535333529202D2070723C
:1023E000696E74206974207769746820273F270D0F
:1023F0000A452078090909656E61626C652F646978
:102400007361626C65206563686F207768656E2014
:10241000747970696E672028783D312F30290D0A54
:102420006520200909097072696E742073746174E3
:102430007573206F6620747970696E6720656368B4
:102440006F0D0A2420780909097072696E74206280
:10245000756666657220636F6E74656E7473206F47
:1024600066206368616E6E656C20782028783D3048
:102470002E2E37290D0A5E2078090909656E6162E2
:102480006C652F64697361626C6520646562756751
:10249000206F75747075742028783D312F30290DA8
:1024A0000A0D0A005245504C592C25642C25632CEA
:1024B0004F4B2C256C640D0A00005245504C592C92
:1024C00025642C25632C4552524F522C256C640DEB
:1024D0000A00D9CFE5FFE1CFD9FF00C0E5FF01C079
:1024E000E5FF02C0E5FF03C0E5FF04C0E5FF05C04E
:1024F000E5FF06C0E5FF07C0E5FF08C0E5FF09C02E
:10250000E5FF0AC0E5FF0BC0E5FF0CC0E5FF0DC00D
:10251000E5FF0EC0E5FF0FC0E5FF10C0E5FF11C0ED
:10252000E5FF12C0E5FF13C0E5FF14C0E5FF15C0CD
:10253000E5FF16C0E5FF17C0E5FF18C0E5FF020E76
:10254000DBCF00F0030EDBCF01F0040EDBCF02F097
:10255000050EDBCF03F0060EDBCF04F0070EDBCF5A
:1025600005F0080EDBCF06F0090EDBCF07F00A0EF0
:10257000DBCF08F0096A0A6A03C0E9FF04C0F3FF71
:10258000055013EC35F00B6E0B50D8B4F0D10B5056
:10259000250A01E0CDD10C6A0D6A0E6A0F6A106A35
:1025A000116A032AD8B0042AD8B0052A03C0E9FF6B
:1025B00004C0F3FF055013EC35F0126E250A15E147
:1025C0001250E56E0250E56E0150E56E0050E56E6A
:1025D000BAEC2BF0040EE126092AD8B00A2A032A05
:1025E000D8B0042AD8B0052AC7D71250750A07E117
:1025F000010E0F6E032AD8B0042AD8B0052A03C0F2
:10260000E9FF04C0F3FF055013EC35F0126E6C0ABD
:1026100008E1010E0C6E032AD8B0042AD8B0052AAE
:102620000AD01250680A07E1010E0E6E032AD8B0D4
:10263000042AD8B0052A03C0E9FF04C0F3FF0550FF
:1026400013EC35F0126E730A03E1010E0D6E3BD0F0
:102650001250640A03E10A0E106E35D01250780A47
:1026600004E1100E106E116A2ED01250580A05E1C6
:10267000100E106E010E116E26D01250630A02E188
:10268000106A21D012506F0A03E1080E106E1BD0A1
:102690001250620A03E1020E106E15D01250E56E60
:1026A0000250E56E0150E56E0050E56EBAEC2BF07D
:1026B000040EE126092AD8B00A2A032AD8B0042A2F
:1026C000D8B0052A59D70D50D8B444D00650030FBE
:1026D0000D6E000E0720126E000E0820136E0DC046
:1026E00006F012C007F013C008F0FD0E0D26FF0E15
:1026F000122213220DC0E9FF12C0F3FF13505CEC4D
:1027000034F00D6EF3CF12F0F4CF13F009C014F0D3
:102710000AC015F00DC0E9FF12C0F3FF135013EC0F
:1027200035F0166E1650D8B413D11650E56E02501F
:10273000E56E0150E56E0050E56EBAEC2BF0040E2C
:10274000E1260D2AD8B0122AD8B0132A142AD8B0FC
:10275000152AE0D70C5023E00650040F0C6E000E33
:1027600007200D6E000E0820126E0CC006F00DC082
:1027700007F012C008F0FC0E0C26FF0E0D221222EC
:102780000CC0E9FF0DC0F3FF125087EC33F00C6E64
:10279000F3CF0DF0F4CF12F0E9CF13F057D00E5075
:1027A0002EE00650020F0E6E000E0720166E000E71
:1027B0000820176E0EC006F016C007F017C008F00C
:1027C000FE0E0E26FF0E162217220EC0E9FF16C0BF
:1027D000F3FF17508EEC34F00E6E0EC00CF00D6A45
:1027E000126A136A0F5032E10C500E6E0EC00CF0DC
:1027F000E86A0EBEFF0E0D6E126E136E27D00650E5
:10280000020F0E6E000E0720166E000E0820176EC7
:102810000EC006F016C007F017C008F0FE0E0E2618
:10282000FF0E162217220EC0E9FF16C0F3FF175045
:102830008EEC34F00E6EF3CF16F00EC00CF016C016
:102840000DF0E86A16BEFF0E126E136E1050D8B46B
:102850005FD00F5013E01050E56E030EE56E700E62
:10286000E56E1350E56E1250E56E0D50E56E0C509E
:10287000E56E7EEC1EF0070EE12612D01050E56EDC
:10288000030EE56E700EE56E1350E56E1250E56EA8
:102890000D50E56E0C50E56EE1EC2DF0070EE126D3
:1028A00009C00EF00AC00FF0700E166E030E176E00
:1028B00016C0E9FF17C0EAFFEFCF18F01850D8B4E0
:1028C0004CD018C010F0115010E01050E56E77ECAD
:1028D00034F0186EE12A185004E0DF0E1014186E60
:1028E00002D010C018F018C010F01050E56E025061
:1028F000E56E0150E56E0050E56EBAEC2BF0040E6B
:10290000E1260E2AD8B00F2A162AD8B0172AD0D717
:102910000C50E56E0250E56E0150E56E0050E56E1C
:10292000BAEC2BF0040EE126092AD8B00A2A19D0F5
:102930000B50E56E0250E56E0150E56E0050E56EFD
:10294000BAEC2BF0040EE126092AD8B00A2A09D0E5
:1029500014C009F015C00AF004D00EC009F00FC071
:102960000AF0032AD8B0042AD8B0052A05D60AC02E
:10297000F3FF0950E4CF18F0E4CF17F0E4CF16F0DE
:10298000E4CF15F0E4CF14F0E4CF13F0E4CF12F06D
:10299000E4CF11F0E4CF10F0E4CF0FF0E4CF0EF06D
:1029A000E4CF0DF0E4CF0CF0E4CF0BF0E4CF0AF06D
:1029B000E4CF09F0E4CF08F0E4CF07F0E4CF06F06D
:1029C000E4CF05F0E4CF04F0E4CF03F0E4CF02F06D
:1029D000E4CF01F0E4CF00F0E4CFD9FF1200D9CF6B
:1029E000E5FFE1CFD9FF00C0E5FF01C0E5FF02C070
:1029F000E5FF03C0E5FF04C0E5FF05C0E5FF06C035
:102A0000E5FF07C0E5FF08C0E5FF09C0E5FF0AC014
:102A1000E5FF0BC0E5FF0CC0E5FF28C3E8FF03019D
:102A2000286B2CC300F003012C6B010EE56E7BECD0
:102A300022F0016EE12A0150D8A42BEF15F0000E10
:102A4000E56E360EE56E2C0EE56E45EC31F0030EAC
:102A5000E126A2EF16F0000EE56E360EE56E4C0E86
:102A6000E56E45EC31F0030EE126026A036A080EBA
:102A7000025CD8B04FEF15F0150E0324046E056A02
:102A8000030E052204C0E9FF05C0EAFF000EEE6E4A
:102A9000000EEF6E032A032A022A37EF15F0020E0A
:102AA0000301286F2BC302F0010E03012B6F036A91
:102AB00003012951035CD8B077EF15F0000EE56EE5
:102AC000780EE56E98EC29F0020EE126046A080EF5
:102AD000045CD8B074EF15F00450E56E5BEC0BF0BD
:102AE000E12A042A67EF15F0032A58EF15F0100EBB
:102AF000036E03C004F003060450D8B403EF16F0CD
:102B0000046A056A080E045CD8B0E8EF15F0010EFF
:102B1000066E000E076E045006E0E86CD89006368C
:102B20000736010FFCE301C008F0096A08500616D9
:102B30000950071606500710D8B4E3EF15F00450FB
:102B4000E56E5BEC0BF0E12A150E0524066E076AB4
:102B5000030E072206C0E9FF07C0EAFFEECF08F028
:102B6000EFCF09F0810E05240A6E0B6A000E0B22CE
:102B70000AC0E9FF0BC0EAFFEECF0AF0EFCF0BF07F
:102B8000010E0B5C02E1F40E0A5CD8B0CAEF15F03E
:102B9000CCEF15F00A6A0B6A0B50E56E0A50E56E31
:102BA0000950E56E0850E56E34EC32F0086EF3CF54
:102BB00009F0040EE12606C0E9FF07C0EAFF08C0DD
:102BC000EEFF09C0EFFF052A052A042A82EF15F05F
:102BD000000EE56EC80EE56E98EC29F0020EE126B7
:102BE00003C004F0056A0550E56E0450E56E000E62
:102BF000E56E360EE56E7C0EE56E45EC31F0050EA9
:102C0000E12679EF15F0036A046A080E035CD8B078
:102C100090EF16F003C005F0066A010E076E000E75
:102C2000086E035006E0E86CD89007360836010FAE
:102C3000FCE301C009F00A6A095007160A50081699
:102C400007500810D8B48BEF16F0150E0424076E49
:102C5000086A030E082207C0E9FF08C0EAFFEECFAA
:102C600009F0EFCF0AF00B6A0C6A0C50E56E0B50BE
:102C7000E56E0A50E56E0950E56E000EE56E000E39
:102C8000E56E000EE56E030EE56E86EC1BF0096E38
:102C9000F3CF0AF0F4CF0BF0E9CF0CF0080EE126E9
:102CA000D8900C320B320A32093207C0E9FF08C053
:102CB000EAFF09C0EEFF0AC0EFFF050E0424096E0B
:102CC0000A6A030E0A2209C0E9FF0AC0EAFFFF0EE2
:102CD000EE6EFF0EEF6E07C0E9FF08C0EAFFEECF11
:102CE00007F0EFCF08F0096A0A6A0A50E56E09504A
:102CF000E56E0850E56E0750E56E0650E56E05502E
:102D0000E56E000EE56E360EE56E820EE56E45EC64
:102D100031F0090EE126042A042A032A05EF16F0F1
:102D2000000EE56E360EE56E8E0EE56E45EC31F06A
:102D3000030EE12603012B6B005003012C6F0250A0
:102D400003012B6FE4CF0CF0E4CF0BF0E4CF0AF0DB
:102D5000E4CF09F0E4CF08F0E4CF07F0E4CF06F0C9
:102D6000E4CF05F0E4CF04F0E4CF03F0E4CF02F0C9
:102D7000E4CF01F0E4CF00F0E4CFD9FF1200D9CFC7
:102D8000E5FFE1CFD9FF00C0E5FF01C0E5FF02C0CC
:102D9000E5FF03C0E5FF04C0E5FF05C0E5FF06C091
:102DA000E5FF07C0E5FF08C0E5FF09C0E5FF0AC071
:102DB000E5FF0BC0E5FF0CC0E5FF0DC0E5FF0EC051
:102DC000E5FF0FC0E5FF10C0E5FF11C0E5FF12C031
:102DD000E5FF13C0E5FF020EDBCF00F0016A026AD7
:102DE000036A046A0050200DF3CF00F0F4CF05F021
:102DF000066A076A086A096A29C30AF00B6A0B5057
:102E0000075C02E10A50065CD8B0DBEF17F0000E59
:102E100000240A6E010E05200B6E29C30CF00D6A0A
:102E200006500C2607500D22FF0E0C26D8A00D06CA
:102E300029C30EF00F6A0F50E56E0E50E56E0D506F
:102E4000E56E0C50E56EA7EC2EF00C6EF3CF0DF096
:102E5000040EE1260D50E56E0C50E56E000EE56E99
:102E6000020EE56EABEC2FF00C6EF3CF0DF0040EFE
:102E7000E1260C500A260D500B220AC0E9FF0BC0B8
:102E8000EAFFEECF0AF0EFCF0BF0000E00240C6E3D
:102E9000010E05200D6E08500C2609500D220CC0A5
:102EA000E9FF0DC0EAFFEECF0CF0EFCF0DF0000E02
:102EB00000240E6E010E05200F6E29C310F0116A5A
:102EC0000650102607501122102AD8B0112A29C303
:102ED00012F0136A1350E56E1250E56E1150E56E54
:102EE0001050E56EA7EC2EF0106EF3CF11F0040E2B
:102EF000E1261150E56E1050E56E000EE56E020EF3
:102F0000E56EABEC2FF0106EF3CF11F0040EE1265E
:102F100010500E2611500F220EC0E9FF0FC0EAFF1D
:102F2000EECF0EF0EFCF0FF00C500A5C106E0D508C
:102F30000B58116E1150E56E1050E56E78EC1AF0DA
:102F4000106EF3CF11F0020EE126000E115C02E1CB
:102F50001F0E105CD8A0C8EF17F00C500E5E0D507D
:102F60000F5A0F50E56E0E50E56E78EC1AF00E6EAB
:102F7000F3CF0FF0020EE126000E0F5C02E11F0EF0
:102F80000E5CD8A0C8EF17F00AC00CF00BC00DF013
:102F90000A6A0B6A0C5001260D5002220A500322C5
:102FA0000B500422020E0826D8B0092A062AD8B0EF
:102FB000072AFCEF16F029C300F0056A066A076AC3
:102FC0000750E56E0650E56E0550E56E0050E56E63
:102FD0000450E56E0350E56E0250E56E0150E56E5B
:102FE00025EC2AF0006EF3CF01F0F4CF02F0E9CF28
:102FF00003F0080EE12601C0F3FF0050E4CF13F008
:10300000E4CF12F0E4CF11F0E4CF10F0E4CF0FF0F2
:10301000E4CF0EF0E4CF0DF0E4CF0CF0E4CF0BF0F2
:10302000E4CF0AF0E4CF09F0E4CF08F0E4CF07F0F2
:10303000E4CF06F0E4CF05F0E4CF04F0E4CF03F0F2
:10304000E4CF02F0E4CF01F0E4CF00F0E4CFD9FF09
:103050001200D9CFE5FFE1CFD9FF00C0E5FF01C0E5
:10306000E5FF02C0E5FF03C0E5FF04C0E5FF05C0C2
:10307000E5FF06C0E5FF07C0E5FF03012E51D8A418
:1030800044EF18F043EF19F00001B1510001B21103
:103090000001B3110001B411D8A457EF18F0D0C04B
:1030A000B1F00001B26B0001B36B0001B46BD0C092
:1030B00000F0016A026A036A0001B151005E00017A
:1030C000B251015A0001B351025A0001B451035ADE
:1030D000000E035C08E1000E025C05E1030E015CDA
:1030E00002E1E90E005CD8A043EF19F0006A016A22
:1030F000080E005CD8B043EF19F061EC35F0026EB9
:10310000010E036E000E046E005006E0E86CD890CD
:1031100003360436010FFCE3056A0250031605501E
:10312000041603500410D8B43EEF19F00050E56EB9
:10313000ABEC2CF0026EF3CF03F0E12AA10E0124D8
:10314000046E056A000E052204C0E9FF05C0EAFF0F
:10315000EECF04F0EFCF05F00350E56E0250E56EC0
:103160000550E56E0450E56EFBEC2FF0046EF3CFD6
:1031700005F0040EE126000E055C02E1060E045C7B
:10318000D8B0EEEF18F0030125510A0F046E000EBF
:1031900003012621056E0350055C02E10250045C28
:1031A000D8B0EEEF18F0B50E0124046E056A000EDB
:1031B000052204C0E9FF05C0EAFFEECF06F0EFCF1D
:1031C00007F0062AD8B0072A04C0E9FF05C0EAFFC5
:1031D00006C0EEFF07C0EFFFFCEF18F0B50E0124AC
:1031E000046E056A000E052204C0E9FF05C0EAFF6F
:1031F000000EEE6E000EEF6ED0C0B1F00001B26BAB
:103200000001B36B0001B46BA10E0124046E056ACA
:10321000000E052204C0E9FF05C0EAFF02C0EEFF70
:1032200003C0EFFFB50E0124026E036A000E0322F5
:1032300002C0E9FF03C0EAFFEECF04F0EFCF05F0D4
:10324000000E055C02E1050E045CD8A03EEF19F00B
:10325000050E0124046E056A030E052204C0E9FF71
:1032600005C0EAFFFF0EEE6EFF0EEF6E02C0E9FF33
:1032700003C0EAFF000EEE6E000EEF6E012A012A77
:10328000002A78EF18F0E4CF07F0E4CF06F0E4CF9F
:1032900005F0E4CF04F0E4CF03F0E4CF02F0E4CF94
:1032A00001F0E4CF00F0E4CFD9FF1200D9CFE5FF61
:1032B000E1CFD9FF00C0E5FF01C0E5FF02C0E5FF97
:1032C00003C0E5FF04C0E5FF05C0E5FF06C0E5FF5C
:1032D00007C0E5FF08C0E5FF09C0E5FF0AC0E5FF3C
:1032E0000BC0E5FF0CC0E5FF0DC0E5FF0EC0E5FF1C
:1032F0000FC0E5FF020EDBCF00F0016A026A036A2D
:10330000046A6AC005F0066A29C307F0086A075014
:103310000526085006226BC007F0086A0750055EB4
:103320000850065A29C307F0086A0850E56E07508E
:10333000E56E0650E56E0550E56E39EC2CF0056E35
:10334000F3CF06F0040EE1260050200DF3CF06F077
:10335000F4CF07F0086A096A05C00AF00B6A0B503F
:10336000095C02E10A50085CD8B00BEF1AF0000EBD
:1033700006240A6E010E07200B6E6AC00CF00D6A5F
:10338000FF0E0C26D8A00D0608500C5E09500D5AF1
:1033900029C30EF00F6A0E500C260F500D2229C3C0
:1033A0000EF00F6A0F50E56E0E50E56E0D50E56E93
:1033B0000C50E56EA7EC2EF00C6EF3CF0DF0040E62
:1033C000E1260D50E56E0C50E56E000EE56E020E26
:1033D000E56EABEC2FF00C6EF3CF0DF0040EE12692
:1033E0000C500A260D500B220AC0E9FF0BC0EAFF61
:1033F000EECF0AF0EFCF0BF00C6A0D6A0A500126EF
:103400000B5002220C5003220D500422082AD8B07F
:10341000092AACEF19F005C006F0076A086A096AC4
:103420000950E56E0850E56E0750E56E0650E56EF2
:103430000450E56E0350E56E0250E56E0150E56EF6
:1034400025EC2AF0016EF3CF02F0F4CF03F0E9CFC0
:1034500004F0080EE12603013051D8B452EF1AF0FF
:103460006BC003F0046A6AC006F0076A086A096A5A
:103470000450E56E0350E56E0750E56E0650E56EAC
:103480000850E56E0550E56E0950E56E0050E56E9A
:10349000000EE56E360EE56EBA0EE56E45EC31F0C7
:1034A0000B0EE12602C0F3FF0150E4CF0FF0E4CF92
:1034B0000EF0E4CF0DF0E4CF0CF0E4CF0BF0E4CF4E
:1034C0000AF0E4CF09F0E4CF08F0E4CF07F0E4CF4E
:1034D00006F0E4CF05F0E4CF04F0E4CF03F0E4CF4E
:1034E00002F0E4CF01F0E4CF00F0E4CFD9FF120006
:1034F000D9CFE5FFE1CFD9FF00C0E5FF01C0E5FF6F
:1035000002C0E5FF03C0E5FF020EDBCF00F0030EB3
:10351000DBCF01F000500110D8B495EF1AF000C0D5
:1035200002F001C003F09BEF1AF0011C036E001CB7
:10353000026E024A032A03C0F3FF0250E4CF03F0F5
:10354000E4CF02F0E4CF01F0E4CF00F0E4CFD9FF04
:10355000120009096164617074697665282564291F
:103560003A2076616C3D20256C642C206176673DA5
:1035700020256C642C206465763D20256C642C200D
:103580006465765F7468723D20256C642C206275DA
:10359000663D202564200D0A000009096164617000
:1035A00074697665282564293A207374616E6461B4
:1035B000726420617665726167650D0A0000090911
:1035C0006164617074697665282564293A206164B4
:1035D0006170746976652061766572616765206DDA
:1035E0006F646520282564290D0A000009092061FF
:1035F00076675B25645D3A20256C64206472696699
:10360000745F6F3A20256C642C20746872313A2004
:10361000256C642C206465763A20256C642C20741B
:103620006872323A20256C640D0A00005741524EF0
:10363000494E473A204E6F2073656E736F72732048
:103640006174746163686564210D0A0043616C698B
:1036500062726174696E672E20506C6561736520BB
:10366000646F206E6F7420746F75636820616E796B
:103670002073656E736F72210D0A000025640D0AB8
:1036800000005B25645D20256C64202000000D0A8D
:10369000000009097365745F7661725F6275665F29
:1036A00073697A653A207661725F6275665F7369E5
:1036B0007A653D202025640D0A0009097661725F54
:1036C00061766572616765282564293A206C656EAC
:1036D0006774683D2025642C20627566706F733AAC
:1036E0002025642C206275665F656E643A2025642F
:1036F0000D0A0000494E464F2C25642C25642C5B96
:1037000000005B005D002000256C6400D9CFE5FF60
:10371000E1CFD9FF00C0E5FF01C0E5FF02C0E5FF32
:1037200003C0E5FF04C0E5FF05C0E5FF06C0E5FFF7
:1037300007C0E5FF020EDBCF00F0030EDBCF01F088
:10374000040EDBCF02F0050EDBCF03F0060EDBCF5D
:1037500004F0070EDBCF05F0080EDBCF06F0090EF4
:10376000DBCF07F000500001F96F0150FA6F0250F3
:10377000FB6F0350FC6F04500301896F05508A6F83
:1037800006508B6F07508C6F0001F95103018B03BA
:10379000F3CF00F0F4CF01F0005003018F6F015020
:1037A000906F0001F95103018903F3CF00F0F4CFCA
:1037B00001F0005003018D6F01508E6F0001FC512C
:1037C00003018903F3CF00F003019051002600505C
:1037D000906F0001FB5103018A03F3CF00F0030156
:1037E000905100260050906F0001FB5103018903A6
:1037F000F3CF00F0F4CF01F003018F510026905178
:10380000012200508F6F0150906F0001FA510301A7
:103810008A03F3CF00F0F4CF01F003018F510026AB
:103820009051012200508F6F0150906F0001FA51AA
:1038300003018B03F3CF00F000500301946F0001EC
:10384000FA5103018903F3CF00F0F4CF01F00050E7
:103850000301926F0150936F0001F95103018C0332
:10386000F3CF00F000500301986F0001F9510301FC
:103870008A03F3CF00F0F4CF01F000500301966FFC
:103880000150976F0301916B0301956B03019151F7
:1038900003018D25006E0301925103018E21016EFB
:1038A0000301935103018F21026E0301945103011F
:1038B0009021036E00508D6F01508E6F02508F6FFC
:1038C0000350906F0301955103018D25006E030194
:1038D000965103018E21016E0301975103018F213F
:1038E000026E0301985103019021036E03C0E9FFAA
:1038F00002C0F4FF01C0F3FF0050E4CF07F0E4CFB3
:1039000006F0E4CF05F0E4CF04F0E4CF03F0E4CF19
:1039100002F0E4CF01F0E4CF00F0E4CFD9FF1200D1
:10392000D9CFE5FFE1CFD9FF00C0E5FF01C0E5FF3A
:1039300002C0E5FF03C0E5FF04C0E5FF05C0E5FFE9
:1039400006C0E5FF07C0E5FF08C0E5FF09C0E5FFC9
:103950000AC0E5FF0BC0E5FF0CC0E5FF0DC0E5FFA9
:103960000EC0E5FF0FC0E5FF10C0E5FF11C0E5FF89
:1039700012C0E5FF13C0E5FF020EDBCF00F003012C
:103980000251D8B467EF1DF000A007D0030103A1D6
:1039900003D08080CDEF1CF0809000A207D00301FF
:1039A00003A303D08082D6EF1CF0809200A407D03E
:1039B000030103A503D08084DFEF1CF0809400A6F0
:1039C00007D0030103A703D08086E8EF1CF08096A0
:1039D00000A807D0030103A903D0808AF1EF1CF0EF
:1039E000809A00AA07D0030103AB03D08282FAEFCA
:1039F0001CF0829200AC07D0030103AD03D0828497
:103A000003EF1DF0829400AE07D0030103AF03D093
:103A100082880CEF1DF0829803013051D8B467EF13
:103A20001DF0016A80B0012A026A036A80B2032A8B
:103A3000046A056A80B4052A066A076A80B6072AFE
:103A4000086A096A80BA092A0A6A0B6A82B20B2AD2
:103A50000C6A0D6A82B40D2A0E6A0F6A82B80F2AA8
:103A6000106A03C311F0126A136A0250E56E015026
:103A7000E56E0450E56E0350E56E0650E56E0550A8
:103A8000E56E0850E56E0750E56E0A50E56E095088
:103A9000E56E0C50E56E0B50E56E0E50E56E0D5068
:103AA000E56E1050E56E0F50E56E1250E56E115048
:103AB000E56E1350E56E0050E56E000EE56E540E97
:103AC000E56E180EE56E45EC31F0170EE126E4CFF9
:103AD00013F0E4CF12F0E4CF11F0E4CF10F0E4CF14
:103AE0000FF0E4CF0EF0E4CF0DF0E4CF0CF0E4CF14
:103AF0000BF0E4CF0AF0E4CF09F0E4CF08F0E4CF14
:103B000007F0E4CF06F0E4CF05F0E4CF04F0E4CF13
:103B100003F0E4CF02F0E4CF01F0E4CF00F0E4CF13
:103B2000D9FF1200D9CFE5FFE1CFD9FF00C0E5FFF3
:103B300001C0E5FF02C0E5FF03C0E5FF04C0E5FFEB
:103B400005C0E5FF06C0E5FF07C0E5FF08C0E5FFCB
:103B500009C0E5FF0AC0E5FF020EDBCF00F061EC13
:103B600035F0016E00C002F0036A030E046E000E11
:103B7000056E005006E0E86CD89004360536010F5B
:103B8000FCE3066A015004160650051604500510A1
:103B9000D8A4CEEF1DF0E86A65EF1EF0010E046EAA
:103BA000000E056E005006E0E86CD890043605362D
:103BB000010FFCE3015004160650051604500510D1
:103BC000D8B419EF1EF00050E56EABEC2CF0046E8B
:103BD000F3CF05F0E12A04C007F005C008F0096A38
:103BE0000A6A0001D351E56E0001D251E56E000171
:103BF000D151E56E0001D051E56E0A50E56E0950D5
:103C0000E56E0850E56E0750E56E0350E56E025014
:103C1000E56E03010151E56E03010051E56E000EF2
:103C2000E56E1D0EE56EFE0EE56E45EC31F00F0EF5
:103C3000E126020E076E000E086E005006E0E86CEA
:103C4000D89007360836010FFCE3075001160850DC
:103C5000061601500610D8B464EF1EF0002A00507A
:103C6000E56EABEC2CF0046EF3CF05F0E12A006AB0
:103C7000016A022AD8B0032A0001D351E56E00017F
:103C8000D251E56E0001D151E56E0001D051E56ED3
:103C90000150E56E0050E56E0550E56E0450E56E8E
:103CA0000350E56E0250E56E03010151E56E03011C
:103CB0000051E56E000EE56E1D0EE56EFE0EE56E22
:103CC00045EC31F00F0EE126010EE4CF0AF0E4CF0F
:103CD00009F0E4CF08F0E4CF07F0E4CF06F0E4CF3A
:103CE00005F0E4CF04F0E4CF03F0E4CF02F0E4CF3A
:103CF00001F0E4CF00F0E4CFD9FF1200D9CFE5FF07
:103D0000E1CFD9FF00C0E5FF01C0E5FF02C0E5FF3C
:103D100003C0E5FF04C0E5FF05C0E5FF06C0E5FF01
:103D200007C0E5FF08C0E5FF09C0E5FF0AC0E5FFE1
:103D30000BC0E5FF0CC0E5FF0DC0E5FF0EC0E5FFC1
:103D40000FC0E5FF020EDBCF00F0030EDBCF01F06A
:103D5000040EDBCF02F0050EDBCF03F0060EDBCF47
:103D600004F0070EDBCF05F0080EDBCF06F0200EC7
:103D7000076E086A06C009F00A6A0B6A0C6AE56AEF
:103D8000E56AE56A0950E56E0350E56E0250E56E9E
:103D90000150E56E0050E56E77EC28F00D6E080ED0
:103DA000E126300E0D263A0E0D5C02E3270E0D269D
:103DB000FF0E0726D8A00806400E07240E6E030E3D
:103DC00008200F6E0EC0E9FF0FC0EAFF0DC0EFFF25
:103DD0000C50E56E0B50E56E0A50E56E0950E56E2D
:103DE0000350E56E0250E56E0150E56E0050E56E41
:103DF00025EC2AF0006EF3CF01F0F4CF02F0E9CF0A
:103E000003F0080EE1260050011002100310D8A4A0
:103E1000B1D707C000F008C001F004C002F005C02F
:103E200003F000C004F001C005F0002AD8B0012A58
:103E3000400E0426030E052204C0E9FF05C0EAFF78
:103E4000EFCF04F002C0E9FF03C0EAFF04C0EFFFB8
:103E5000022AD8B0032A000E015C02E1200E005CA9
:103E6000E0E302C0E9FF03C0EAFF000EEF6AE4CF1F
:103E70000FF0E4CF0EF0E4CF0DF0E4CF0CF0E4CF80
:103E80000BF0E4CF0AF0E4CF09F0E4CF08F0E4CF80
:103E900007F0E4CF06F0E4CF05F0E4CF04F0E4CF80
:103EA00003F0E4CF02F0E4CF01F0E4CF00F0E4CF80
:103EB000D9FF12000001686B39EC2BF0F0EC32F006
:103EC000070EE56ED00EE56EFCEC31F0020EE12639
:103ED00003013051D8B477EF1FF0000EE56E4F0E9E
:103EE000E56EEE0EE56E45EC31F0030EE126E5ECF5
:103EF00033F003013051D8B488EF1FF0000EE56EA7
:103F0000500EE56E000EE56E45EC31F0030EE12635
:103F1000A4EC34F003013051D8B499EF1FF0000E37
:103F2000E56E500EE56E140EE56E45EC31F0030EB5
:103F3000E12624EC35F028EC20F0000EE56E500E62
:103F4000E56E2A0EE56E45EC31F0030EE126000E1B
:103F5000E56E500EE56E4E0EE56E000EE56E500EEF
:103F6000E56E480EE56E000EE56E500EE56E2E0E07
:103F7000E56E45EC31F0090EE126000EE56E500EBF
:103F8000E56E5C0EE56E45EC31F0030EE126000EA9
:103F9000E56E500EE56E900EE56E45EC31F0030EC9
:103FA000E126000EE56E500EE56E2A0EE56E45EC3C
:103FB00031F0030EE126EFEC14F0000EE56E500E2A
:103FC000E56EB40EE56E45EC31F0030EE126000E11
:103FD000E56E020EE56E98EC29F0020EE126030173
:103FE0002B51D8B418EF20F0000164510001601982
:103FF00011E100016551000161190CE100016651F8
:104000000001621907E1000167510001631902E133
:1040100018EF20F00301A251E56E92EC1DF0E12AA9
:1040200064C060F065C061F066C062F067C063F0B4
:104030003FEC34F0DFEC27F015EC00F029EC18F041
:1040400000016851D8B4E7EF1FF05AEF1FF01200DB
:10405000D9CFE5FFE1CFD9FF00C0E5FF01C0E5FF03
:1040600002C0E5FF03C0E5FF04C0E5FF05C0E5FFB2
:10407000CE0E0001D86F500E0001D96F000E000166
:10408000DA6FD40E0001DB6F500E0001DC6F000E02
:104090000001DD6FD60E0001DE6F500E0001DF6FF4
:1040A000000E0001E06FD80E0001E16F500E00011C
:1040B000E26F000E0001E36FDA0E0001E46F500EB4
:1040C0000001E56F000E0001E66FDC0E0001E76FF6
:1040D000500E0001E86F000E0001E96FD60E0001DE
:1040E000EA6F500E0001EB6F000E0001EC6FDE0E68
:1040F0000001ED6F500E0001EE6F000E0001EF6F3A
:10410000E00E0001F06F500E0001F16F000E000193
:10411000F26FE20E0001F36F500E0001F46F000E1B
:104120000001F56FE80E0001F66F500E0001F76F09
:10413000000E0001F86F006A016AD80E0124026EB9
:10414000036A000E032202C0E9FF03C0EAFFEECFBC
:1041500002F0EECF03F0EFCF04F002C0E9FF03C09E
:10416000F3FF045013EC35F0056E0550250A02E10B
:10417000D7EF20F00450E56E0350E56E0250E56E77
:10418000000EE56E500EE56EEA0EE56E45EC31F080
:10419000060EE126030E0126002A000EE56E640ECF
:1041A000E56E98EC29F0020EE1269DEF20F0000E5E
:1041B000E56E500EE56E2A0EE56E45EC31F0030E0D
:1041C000E126E4CF05F0E4CF04F0E4CF03F0E4CF40
:1041D00002F0E4CF01F0E4CF00F0E4CFD9FF120009
:1041E000D9CFE5FFE1CFD9FF00C0E5FF01C0E5FF72
:1041F00002C0E5FF03C0E5FF04C0E5FF05C0E5FF21
:1042000006C0E5FF07C0E5FF08C0E5FF09C0E5FF00
:10421000020EDBCF00F0030EDBCF01F0040EDBCF8C
:1042200002F0036A046A056A00C006F001C007F0E4
:1042300002C008F006C0E9FF07C0F3FF085013EC06
:1042400035F0096E09501BE00950800F460F04E25B
:104250000950800F500F13E206C0E9FF07C0F3FFBB
:10426000085013EC35F0096E2D0A09E009502B0AAD
:1042700006E0062AD8B0072AD8B0082ADBD706C03D
:1042800000F007C001F008C002F006C0E9FF07C057
:10429000F3FF085013EC35F0066E076A2D0A01E1B2
:1042A000072A075002E0010E056E075003E1065091
:1042B0002B0A05E1002AD8B0012AD8B0022A00C092
:1042C000E9FF01C0F3FF025013EC35F0066E065013
:1042D00029E00650800F500F25E30650800F460F4F
:1042E00021E20450E56E0350E56EE56A0A0EE56EC4
:1042F000ABEC2FF0076EF3CF08F0040EE126096A4D
:1043000006BE0968D00E0626D8A009060650072466
:10431000036E09500820046E002AD8B0012AD8B0D4
:10432000022ACDD705500AE0041C016E031C006E62
:10433000004A012A01C0F3FF005003D004C0F3FF7C
:104340000350E4CF09F0E4CF08F0E4CF07F0E4CF66
:1043500006F0E4CF05F0E4CF04F0E4CF03F0E4CFBF
:1043600002F0E4CF01F0E4CF00F0E4CFD9FF120077
:10437000E8CFE5FFD8CFE5FFE0CFE5FFF3CFE5FFDE
:10438000F4CFE5FFE9CFE5FFEACFE5FFFACFE5FFA0
:10439000FBCFE5FFD9CFE5FFE1CFD9FF00C0E5FFB7
:1043A00001C0E5FF02C0E5FF9EA2E6EF21F09E926C
:1043B0000001D02BD8A002D00001D12BD8A002D070
:1043C0000001D22BD8A002D00001D32B9EAA60EF0F
:1043D00022F0CCEC34F00301A56F0001D451800F22
:1043E000720FD8B02FEF22F00301A551800F600F9C
:1043F000D8A02FEF22F00301A551800F010FD8B0F4
:104400002FEF22F003012F51D8B41BEF22F0A5C3E8
:1044100000F0016A0301A5BF01680150E56E00507C
:10442000E56E000EE56E5E0EE56EAE0EE56E45ECD9
:1044300031F0050EE126600E0001D425006E016A00
:104440000001D4BF0168030E0122A5C302F000C021
:10445000E9FF01C0EAFF02C0EFFF0001D42B030116
:10446000A5510A0A02E140EF22F00301A5510D0A0D
:1044700002E140EF22F00301A551D8A45FEF22F042
:10448000600E0001D425006E016A0001D4BF0168EE
:10449000030E012200C0E9FF01C0EAFF000EEF6E2B
:1044A000010E0001CF6F0001D46B000EE56E5E0EB1
:1044B000E56EB20EE56E45EC31F0030EE1269E9AF4
:1044C000E4CF02F0E4CF01F0E4CF00F0E4CFD9FF75
:1044D000E4CFFBFFE4CFFAFFE4CFEAFFE4CFE9FF4C
:1044E000E4CFF4FFE4CFF3FFE4CFE0FFE4CFD8FF65
:1044F000E4CFE8FF1000D9CFE5FFE1CFD9FF00C03E
:10450000E5FF01C0E5FF02C0E5FF03C0E5FF04C011
:10451000E5FF05C0E5FF06C0E5FF07C0E5FF08C0F1
:10452000E5FF09C0E5FF0AC0E5FF020EDBCF00F0A2
:10453000016A2BC302F061EC35F0036EFF0EE56EED
:10454000E0EC34F0E12A010E03012B6F010EE56E61
:10455000F40EE56E98EC29F0020EE126000EE56EF1
:10456000650EE56E120EE56E45EC31F0030EE126A8
:10457000046A080E045CD8B0FEEF22F00450E56E29
:10458000ABEC2CF0056EF3CF06F0E12A076A086A5F
:104590000850800F800F08E1000E075C05E1FE0E59
:1045A000065C02E1D30E055CD8B0FBEF22F0010EF1
:1045B000096E045005E0E86CD8900936010FFDE360
:1045C0000950011204C009F00A6A0850E56E07504C
:1045D000E56E0650E56E0550E56E0A50E56E095031
:1045E000E56E000EE56E650EE56E240EE56E45EC9B
:1045F00031F0090EE126042AB9EF22F0000EE56E33
:10460000650EE56E300EE56E45EC31F0030EE126E9
:104610000050D8B416EF23F00150E56EE0EC34F012
:10462000E12A010E03012B6F1EEF23F00350E56E0C
:10463000E0EC34F0E12A025003012B6F0150E4CF8B
:104640000AF0E4CF09F0E4CF08F0E4CF07F0E4CFBC
:1046500006F0E4CF05F0E4CF04F0E4CF03F0E4CFBC
:1046600002F0E4CF01F0E4CF00F0E4CFD9FF120074
:10467000D9CFE5FFE1CFD9FF00C0E5FF030102512B
:10468000D8B4E6EF23F0030104A110D0006A80B093
:10469000002A0050D880E866D890006A00360050A2
:1046A000010BF46E8050FE0BF410806E030104A326
:1046B00011D0006A80B2002A0050D880E866D890F5
:1046C000006A00360050010BE844F46E8050FD0B88
:1046D000F410806E030104A512D0006A80B4002A91
:1046E0000050D880E866D890006A00360050010B70
:1046F000E844E844F46E8050FB0BF410806E030134
:1047000004A712D0006A80B6002A0050D880E8665C
:10471000D890006A00360050010BE838E840F46E8B
:104720008050F70BF410806E030104A912D0006AC8
:1047300080BA002A0050D880E866D890006A003617
:104740000050010BE838E844F46E8050DF0BF410A1
:10475000806E030104AB11D0006A82B2002A0050BF
:10476000D880E866D890006A00360050010BE84413
:10477000F46E8250FD0BF410826E030104AD12D072
:10478000006A82B4002A0050D880E866D890006A97
:1047900000360050010BE844E844F46E8250FB0BF5
:1047A000F410826E030104AF11D0006A82B8002AAF
:1047B0000050D880E866D890006A00360050010B9F
:1047C000E838F46E8250EF0BF410826EE4CF00F004
:1047D000E4CFD9FF1200D9CFE5FFE1CFD9FF00C068
:1047E000E5FF01C0E5FF02C0E5FF03C0E5FF04C02F
:1047F000E5FF05C0E5FF06C0E5FF07C0E5FF08C00F
:10480000E5FF09C0E5FF020EDBCF00F0030EDBCFB2
:1048100001F0026A036A0350800F800F02E1080E64
:10482000025CD8B056EF24F00250046E0450070822
:10483000046E056A04BE0568800E0426030E052278
:10484000010E066E000E076E02500FE007E6E86CE0
:10485000D89006360736010FFCE307D0D89007BE84
:10486000D88007320632010FFAE300C008F0096A67
:1048700008500616095007160750800F800F02E1F6
:10488000010E065CD8A049EF24F0310E066E4BEF06
:1048900024F0300E066E04C0E9FF05C0EAFF06C032
:1048A000EFFF022AD8B0032A0BEF24F00301886B34
:1048B000030E026E800E006E800E036E046A01BE4F
:1048C00004680001D351E56E0001D251E56E00018C
:1048D000D151E56E0001D051E56E0350E56E0250F6
:1048E000E56E0050E56E0450E56E0150E56E030183
:1048F0000151E56E03010051E56E000EE56E1D0EDF
:10490000E56EEA0EE56E45EC31F00E0EE126E4CFE1
:1049100009F0E4CF08F0E4CF07F0E4CF06F0E4CFED
:1049200005F0E4CF04F0E4CF03F0E4CF02F0E4CFED
:1049300001F0E4CF00F0E4CFD9FF1200D9CFE5FFBA
:10494000E1CFD9FF00C0E5FF01C0E5FF02C0E5FFF0
:1049500003C0E5FF04C0E5FF05C0E5FFD59ECD908F
:104960008184818A00016951200DF3CF00F0F4CFDA
:1049700001F0000E0026010E0122D89000016A35D8
:10498000026E02500026E86A0122D6CF02F0036AC6
:10499000D7CF04F0056A0550E56E0450E56E010EB0
:1049A000E56E000EE56EABEC2FF0046EF3CF05F074
:1049B000040EE1260450022605500322046A056A0B
:1049C0000250FF08026EFF0E0356000E0456000E42
:1049D000055600C0E9FF01C0EAFF02C0EEFF03C0B8
:1049E000EFFF00016929006E0050200DF3CF00F0A9
:1049F000F4CF01F0000E0026010E0122D890000134
:104A00006A35026E02500026E86A0122CECF02F01B
:104A1000036ACFCF04F0056A0550E56E0450E56ED9
:104A2000010EE56E000EE56EABEC2FF0046EF3CFD9
:104A300005F0040EE1260450022605500322046A04
:104A4000056A0250FF08026EFF0E0356000E045660
:104A5000000E055600C0E9FF01C0EAFF02C0EEFFEC
:104A600003C0EFFF69C000F0D58ECD80B2EC2AF014
:104A7000D76AD66ACF6ACE6A8194819A0050E4CF11
:104A800005F0E4CF04F0E4CF03F0E4CF02F0E4CF8C
:104A900001F0E4CF00F0E4CFD9FF1200D9CFE5FF59
:104AA000E1CFD9FF00C0E5FF01C0E5FF02C0E5FF8F
:104AB00003C0E5FF04C0E5FF05C0E5FF020EDBCF44
:104AC00000F000C001F0026A0250E56E0150E56E90
:104AD00003010151E56E03010051E56E000EE56E24
:104AE000360EE56EF40EE56E45EC31F0070EE1266C
:104AF0000050200DF3CF00F0F4CF01F0026A036AFA
:104B000003012951025CD8B0DDEF25F0025000010D
:104B10006B1902E18EEF25F09AEF25F0000EE56E9D
:104B2000370EE56E020EE56E45EC31F0030EE12620
:104B3000B8EF25F0025000016A1902E1A2EF25F05A
:104B4000AEEF25F0000EE56E370EE56E040EE56E55
:104B500045EC31F0030EE126B8EF25F0000EE56ECE
:104B6000370EE56E060EE56E45EC31F0030EE126DC
:104B7000000E0024046E010E0120056E0350042671
:104B8000E86A052204C0E9FF05C0EAFFEECF04F0A1
:104B9000EFCF05F00550E56E0450E56E000EE56EB2
:104BA000370EE56E080EE56E45EC31F0050EE12698
:104BB000032A032A022A80EF25F0000EE56E360E46
:104BC000E56E8E0EE56E45EC31F0030EE126E4CF86
:104BD00005F0E4CF04F0E4CF03F0E4CF02F0E4CF3B
:104BE00001F0E4CF00F0E4CFD9FF1200D9CFE5FF08
:104BF000E1CFD9FF00C0E5FF01C0E5FF02C0E5FF3E
:104C000003C0E5FF020EDBCF69F0010E006E010E5E
:104C1000016E030E026E0001695105E0E86CD89048
:104C20000236010FFDE3030127510216550E02144F
:104C3000036E0350010A02E12FEF26F00350040A2D
:104C400002E134EF26F00350100A02E139EF26F0BA
:104C50000350400A02E13EEF26F043EF26F0819038
:104C60008192006A44EF26F081808192006A44EFCD
:104C700026F081908182006A44EF26F08180818253
:104C8000006A44EF26F08184AA0E02160250020A3E
:104C900002E15CEF26F00250080A02E161EF26F023
:104CA0000250200A02E166EF26F00250800A02E17B
:104CB0006BEF26F070EF26F081968198016A71EF14
:104CC00026F081868198016A71EF26F081968188AD
:104CD000016A71EF26F081868188016A71EF26F002
:104CE000818A0050010BE844E844F46E8150FB0BCC
:104CF000F410816E0150010BE838E844F46E8150E5
:104D0000DF0BF410816E006A81BA002A005002089D
:104D1000006E016A81B4012A0150005E0050E4CFA8
:104D200003F0E4CF02F0E4CF01F0E4CF00F0E4CFF1
:104D3000D9FF1200D9CFE5FFE1CFD9FF00C0E5FFD1
:104D400001C0E5FF02C0E5FF03C0E5FF04C0E5FFC9
:104D500005C0E5FF06C0E5FF07C0E5FF08C0E5FFA9
:104D600009C0E5FF0AC0E5FF0BC0E5FF0CC0E5FF89
:104D70000DC0E5FF020EDBCF00F0016A026A036A94
:104D8000046A0050200DF3CF00F0F4CF05F0066A5E
:104D9000076A086A096A29C30AF00B6A0B50075CA4
:104DA00002E10A50065CD8B0FBEF26F0000E0024AA
:104DB0000A6E010E05200B6E08500A2609500B22C0
:104DC0000AC0E9FF0BC0EAFFEECF0AF0EFCF0BF00D
:104DD0000C6A0D6A0A5001260B5002220C50032265
:104DE0000D500422020E0826D8B0092A062AD8B08F
:104DF000072ACBEF26F029C300F0056A066A076A86
:104E00000750E56E0650E56E0550E56E0050E56E04
:104E10000450E56E0350E56E0250E56E0150E56EFC
:104E200025EC2AF0006EF3CF01F0F4CF02F0E9CFC9
:104E300003F0080EE12601C0F3FF0050E4CF0DF0AF
:104E4000E4CF0CF0E4CF0BF0E4CF0AF0E4CF09F0AC
:104E5000E4CF08F0E4CF07F0E4CF06F0E4CF05F0AC
:104E6000E4CF04F0E4CF03F0E4CF02F0E4CF01F0AC
:104E7000E4CF00F0E4CFD9FF1200D9CFE5FFE1CFB6
:104E8000D9FF00C0E5FF01C0E5FF02C0E5FF03C098
:104E9000E5FF04C0E5FF05C0E5FF000EE56E4F0E1F
:104EA000E56E460EE56E45EC31F0030EE126006A34
:104EB000016A000E015C02E1400E005CD8B08AEF8E
:104EC00027F0000EE56E4F0EE56E620EE56E45ECC6
:104ED00031F0030EE1260050026E000E0024036E36
:104EE000030E0120046E0450046E0350036E800E06
:104EF000056E0550E56E0450E56E0350E56E0250F8
:104F0000E56EC4EC30F0040EE126002AD8B0012A88
:104F100059EF27F0000EE56E4F0EE56E640EE56E5C
:104F200045EC31F0030EE126E4CF05F0E4CF04F0C8
:104F3000E4CF03F0E4CF02F0E4CF01F0E4CF00F0DF
:104F4000E4CFD9FF1200536176696E6720636F6EFC
:104F500066696720746F20454550524F4D3A0D0ADF
:104F600000002E0020646F6E650D0A005265737498
:104F70006F72696E6720636F6E6669672066726F15
:104F80006D20454550524F4D3A0D0A003D3D3D3D87
:104F90003D3D3D3D3D3D3D3D3D3D3D3D3D3D0D0AA4
:104FA0000000257800000D0A3D3D3D3D3D3D3D3D65
:104FB0003D3D3D3D3D3D3D3D3D3D0D0A0000D9CFD0
:104FC000E5FFE1CFD9FF82BAF4EF27F0F29E000EA1
:104FD000E56E500EE56EBC0EE56E45EC31F0030E4D
:104FE000E126EFEC14F0F28EE4CFD9FF1200696EE7
:104FF00069742074696D6572732E2E2E0D0A00007F
:10500000696E697420636F756E746572732E2E2ECF
:105010000D0A0000696E697420696E74657272759C
:105020007074732E2E2E0D0A00000D0A00004361CD
:1050300070426F617264202573202D204275696C67
:10504000643A2025730D0A0076322E30000032308B
:105050003038313030365F31343237002863292020
:1050600032303038205261706861656C2057696D4C
:105070006D65722C20687474703A2F2F7777772EB5
:1050800063617073656E73652E6F72670D0A000041
:105090007479706520273F203C454E5445523E2789
:1050A00020666F7220636F6D6D616E642068656C41
:1050B000700D0A0052454144590D0A00427574743E
:1050C0006F6E2070726573736564210D0A001B5B3F
:1050D000316D000043006100700042006F007200FB
:1050E00064001B5B306D0000250025730000D9CFE4
:1050F000E5FFE1CFD9FF00C0E5FF01C0E5FF02C039
:10510000E5FF03C0E5FF04C0E5FF05C0E5FF06C0FD
:10511000E5FF07C0E5FF08C0E5FF09C0E5FF0AC0DD
:10512000E5FF020EDBCF00F0030EDBCF01F0040E33
:10513000DBCF02F0050EDBCF03F0060EDBCF04F071
:10514000070EDBCF05F0080EDBCF06F0090EDBCF34
:1051500007F0086A096A07340A6A0A360AB01BD0DF
:10516000045004260536063607360750035C08E16E
:105170000650025C05E10550015C02E10450005C50
:1051800006E2D890073206320532043204D0092AEA
:1051900009C008F0E0D70750035C08E10650025C44
:1051A00005E10550015C02E10450005C08E3045095
:1051B000005E0550015A0650025A0750035AD89013
:1051C000073206320532043208C009F008060950D9
:1051D000E2E103C0E9FF02C0F4FF01C0F3FF0050A9
:1051E000E4CF0AF0E4CF09F0E4CF08F0E4CF07F011
:1051F000E4CF06F0E4CF05F0E4CF04F0E4CF03F011
:10520000E4CF02F0E4CF01F0E4CF00F0E4CFD9FF27
:105210001200D9CFE5FFE1CFD9FF00C0E5FF01C003
:10522000E5FF02C0E5FF03C0E5FF04C0E5FF05C0E0
:10523000E5FF020EDBCF00F0080E005CD8A025EFE2
:1052400029F0F36AE86A89EF29F0010E016E000E79
:10525000026E005006E0E86CD89001360236010F6D
:10526000FCE327C303F0046A03500116045002163E
:1052700001500210D8A441EF29F0F36AE86A89EFDF
:1052800029F00050200DF3CF00F0F4CF01F0000E14
:105290000026010E01226AC002F0036A29C304F04D
:1052A000056A0450022605500322FF0E0226D8A0EC
:1052B000030629C304F0056A0550E56E0450E56E47
:1052C0000350E56E0250E56E39EC2CF0026EF3CF20
:1052D00003F0040EE1260350E56E0250E56E000E69
:1052E000E56E020EE56EABEC2FF0026EF3CF03F02D
:1052F000040EE126025000260350012200C0E9FFFF
:1053000001C0EAFFEECF00F0EFCF01F001C0F3FFE4
:105310000050E4CF05F0E4CF04F0E4CF03F0E4CF95
:1053200002F0E4CF01F0E4CF00F0E4CFD9FF1200A7
:10533000D9CFE5FFE1CFD9FF00C0E5FF01C0E5FF10
:1053400002C0E5FF03C0E5FF04C0E5FF05C0E5FFBF
:1053500006C0E5FF07C0E5FF08C0E5FF09C0E5FF9F
:105360000AC0E5FF0BC0E5FF0CC0E5FF0DC0E5FF7F
:10537000020EDBCF00F0030EDBCF01F0D0C002F055
:10538000D1C003F0D2C004F0D3C005F00250000138
:10539000D05D066E03500001D159076E0450000124
:1053A000D259086E05500001D359096E00C00AF0A9
:1053B00001C00BF00C6A0D6A0D50095C08E10C503D
:1053C000085C05E10B50075C02E10A50065CD8B0AE
:1053D000EDEF29F00000C6EF29F0E4CF0DF0E4CFA7
:1053E0000CF0E4CF0BF0E4CF0AF0E4CF09F0E4CF07
:1053F00008F0E4CF07F0E4CF06F0E4CF05F0E4CF07
:1054000004F0E4CF03F0E4CF02F0E4CF01F0E4CF06
:1054100000F0E4CFD9FF12007570646174655F6CB1
:1054200065645F7374617465282578292028626D2E
:105430003A2578293A202564256425642564256465
:105440002564256425640D0A0000D9CFE5FFE1CF6E
:10545000D9FF00C0E5FF01C0E5FF02C0E5FF03C0C2
:10546000E5FF04C0E5FF05C0E5FF06C0E5FF07C096
:10547000E5FF08C0E5FF09C0E5FF0AC0E5FF0BC076
:10548000E5FF0CC0E5FF0DC0E5FF020EDBCF00F02D
:10549000030EDBCF01F0040EDBCF02F0050EDBCFF5
:1054A00003F0060EDBCF04F0070EDBCF05F0080E8D
:1054B000DBCF06F0090EDBCF07F0086A096A0A6A3B
:1054C0000B6A200E0C6E03340D6A0D36010E0D169C
:1054D00000500026013602360336085008260936E9
:1054E0000A360B360D50D8A4088007500B5C08E133
:1054F00006500A5C05E10550095C02E10450085CB5
:1055000009E30450085E0550095A06500A5A07502C
:105510000B5A00800C2ED7D703C0E9FF02C0F4FF5E
:1055200001C0F3FF0050E4CF0DF0E4CF0CF0E4CF66
:105530000BF0E4CF0AF0E4CF09F0E4CF08F0E4CFB9
:1055400007F0E4CF06F0E4CF05F0E4CF04F0E4CFB9
:1055500003F0E4CF02F0E4CF01F0E4CF00F0E4CFB9
:10556000D9FF1200D9CFE5FFE1CFD9FF00C0E5FF99
:1055700001C0E5FF02C0E5FF03C0E5FF04C0E5FF91
:10558000006A03012751D8B42CEF2BF00050D8A4A7
:105590002CEF2BF00001692B0001692B070E000195
:1055A000695DD8A022EF2BF00001696B00016A2B26
:1055B0000301295100016A5DD8A0E1EF2AF0000142
:1055C0006A6B6AC001F0026AFF0E0126D8A00206CB
:1055D0006BC003F0046A0350015E0450025A29C3F1
:1055E00003F0046A035001260450022229C303F089
:1055F000046A0450E56E0350E56E0250E56E0150FA
:10560000E56E39EC2CF0016EF3CF02F0040EE126CA
:105610006CC003F0046A0250800FF36E0450800FD8
:10562000F35C02E10350015CD8A022EF2BF00001F3
:105630006B2B0301295100016B5DD8A022EF2BF0E9
:1056400000016B6B69C001F00150E56EF6EC25F0CE
:10565000006EE12AC6EF2AF0E4CF04F0E4CF03F0B5
:10566000E4CF02F0E4CF01F0E4CF00F0E4CFD9FFC3
:105670001200D9CFE5FFE1CFD9FF00C0E5FF01C09F
:10568000E5FF02C0E5FF03C0E5FF04C0E5FF05C07C
:10569000E5FF0301006B0301016B010E0301026FC3
:1056A0000301036B0301046B006A016A026A036A67
:1056B0000150800F800F02E1080E005CD8B086EF29
:1056C0002BF0050E0224046E030E0320056E04C0A9
:1056D000E9FF05C0EAFF000EEE6E000EEF6E150E3C
:1056E0000224046E030E0320056E04C0E9FF05C00A
:1056F000EAFF000EEE6E000EEF6E020E0226D8B02C
:10570000032A002AD8B0012A58EF2BF00301256B99
:105710000301266B0301276B020E0301286F100E95
:105720000301296F000EE56E0F0EE56E82EC30F07E
:10573000020EE126010E03012B6F010E03012C6FF7
:10574000010E03012D6F010E03012E6F010E0301E7
:105750002F6F0301306BE4CF05F0E4CF04F0E4CF0A
:1057600003F0E4CF02F0E4CF01F0E4CF00F0E4CFA7
:10577000D9FF1200D9CFE5FFE1CFD9FF00C0E5FF87
:1057800001C0E5FF02C0E5FF03C0E5FF04C0E5FF7F
:1057900005C0E5FF06C0E5FF07C0E5FF020EDBCF51
:1057A00000F0030EDBCF01F0040EDBCF02F0050E9C
:1057B000DBCF03F002C006F00650046E800A28E139
:1057C00000C0E9FF01C0F3FF02505CEC34F0056E4D
:1057D000F3CF06F0F4CF07F003C0E5FF05C0E9FF03
:1057E00006C0F3FF07504EEC35F0052AD8B0062A64
:1057F000D8B0072A05C0E5FF06C0F4FF07C0F6FFD2
:1058000000C0E9FF01C0F3FF025034EC35F01ED0B8
:1058100004AA1CD0200E041A045004E103508BEC9F
:1058200035F014D00450010A04E1035092EC35F035
:105830000DD004500F0A04E103507CEC35F006D083
:1058400004500E0A03E103508FEC35F0E4CF07F06B
:10585000E4CF06F0E4CF05F0E4CF04F0E4CF03F0AA
:10586000E4CF02F0E4CF01F0E4CF00F0E4CFD9FFC1
:105870001200D9CFE5FFE1CFD9FF00C0E5FF01C09D
:10588000E5FF02C0E5FF03C0E5FF04C0E5FF05C07A
:10589000E5FF06C0E5FF020EDBCF00F0030EDBCF15
:1058A00001F0040EDBCF02F0050EDBCF03F0D88051
:1058B00001AED890046A0436045007E0011C066E5D
:1058C000001C056E054A062A04D000C005F001C080
:1058D00006F005C000F006C001F0D88003AED890F5
:1058E00007E3031C066E021C056E054A062A04D057
:1058F00002C005F003C006F00650E56E0550E56EE7
:105900000150E56E0050E56EA7EC2EF0006EF3CF6F
:1059100001F0040EE12604500AE0011C036E001C95
:10592000026E024A032A03C0F3FF025003D001C0F3
:10593000F3FF0050E4CF06F0E4CF05F0E4CF04F02D
:10594000E4CF03F0E4CF02F0E4CF01F0E4CF00F0C5
:10595000E4CFD9FF1200D9CFE5FFE1CFD9FF00C0D6
:10596000E5FF01C0E5FF02C0E5FF020EDBCF00F05E
:1059700003012851D8A4CAEF2CF00050E56E09ECC1
:1059800029F0016EF3CF02F0E12A02C0F3FF0150CB
:105990000BEF2DF003012851020A02E1D2EF2CF0A7
:1059A000DFEF2CF00050E56E5BEC0BF0016EF3CFF7
:1059B00002F0E12A02C0F3FF01500BEF2DF00301CA
:1059C0002851010A02E1E7EF2CF0F4EF2CF000502F
:1059D000E56E9AEC26F0016EF3CF02F0E12A02C0E8
:1059E000F3FF01500BEF2DF003012851030A02E1F0
:1059F000FCEF2CF009EF2DF00050E56EBFEC16F037
:105A0000006EF3CF01F0E12A01C0F3FF00500BEF6D
:105A10002DF0F36AE86AE4CF02F0E4CF01F0E4CFBE
:105A200000F0E4CFD9FF1200D9CFE5FFE1CFD9FFD5
:105A300000C0E5FF01C0E5FF02C0E5FF03C0E5FFD0
:105A400004C0E5FF05C0E5FF000EE56E4F0EE56EF4
:105A50008C0EE56E45EC31F0030EE126006A016A1A
:105A6000000E015C02E1400E005CD8B062EF2DF048
:105A70000050026E030E046EA40E036E800E056EBF
:105A80000550E56E0450E56E0350E56E0250E56E7C
:105A9000C5EC32F0040EE126A4C302F0036A035001
:105AA000E56E0250E56E000EE56E4F0EE56EA20E3D
:105AB000E56E45EC31F0050EE126002AD8B0012A4A
:105AC00030EF2DF0000EE56E4F0EE56EA60EE56E82
:105AD00045EC31F0030EE126E4CF05F0E4CF04F00D
:105AE000E4CF03F0E4CF02F0E4CF01F0E4CF00F024
:105AF000E4CFD9FF1200D9CFE5FFE1CFD9FF00C035
:105B0000E5FF01C0E5FF02C0E5FF03C0E5FF04C0FB
:105B1000E5FF05C0E5FF000EE56E4F0EE56E6C0E6D
:105B2000E56E45EC31F0030EE126006A016A000ED5
:105B3000015C02E1400E005CD8B0C8EF2DF0000E11
:105B4000E56E4F0EE56E620EE56E45EC31F0030E2C
:105B5000E1260050026E000E0024036E030E0120A9
:105B6000046E0450046E0350036E800E056E0550E3
:105B7000E56E0450E56E0350E56E0250E56EC5EC2F
:105B800032F0040EE126002AD8B0012A97EF2DF05A
:105B9000000EE56E4F0EE56E640EE56E45EC31F0DD
:105BA000030EE126E4CF05F0E4CF04F0E4CF03F0E8
:105BB000E4CF02F0E4CF01F0E4CF00F0E4CFD9FF6E
:105BC0001200D9CFE5FFE1CFD9FF00C0E5FF01C04A
:105BD000E5FF02C0E5FF03C0E5FF04C0E5FF05C027
:105BE000E5FF06C0E5FF020EDBCF00F0030EDBCFC2
:105BF00001F0040EDBCF02F0050EDBCF03F0060E42
:105C0000DBCF04F0070EDBCF05F0080EDBCF06F08C
:105C1000D88003AED89016E306500A0A13E104C0F8
:105C2000E9FF05C0EAFF2D0EEF6E042AD8B0052A61
:105C3000031E021E011E006C05E1012A03E1022A77
:105C4000D8B4032A0650E56E0550E56E0450E56EA3
:105C50000350E56E0250E56E0150E56E0050E56EB2
:105C60007EEC1EF0070EE126E4CF06F0E4CF05F04F
:105C7000E4CF04F0E4CF03F0E4CF02F0E4CF01F08E
:105C8000E4CF00F0E4CFD9FF1200D9CFE5FFE1CF98
:105C9000D9FF00C0E5FF01C0E5FF02C0E5FF03C07A
:105CA000E5FF04C0E5FF020EDBCF00F000016C5100
:105CB000005CD8B082EF2EF06AC001F0026A00C02A
:105CC00003F0046A0350015E0450025A29C303F032
:105CD000046A035001260450022229C303F0046A17
:105CE0000450E56E0350E56E0250E56E0150E56E1E
:105CF00039EC2CF0016EF3CF02F0040EE1260150D6
:105D000000016B6F00C06CF003013051D8B49AEF02
:105D10002EF06CC000F0016A0150E56E0050E56E97
:105D2000000EE56E360EE56E920EE56E45EC31F036
:105D3000050EE126E4CF04F0E4CF03F0E4CF02F057
:105D4000E4CF01F0E4CF00F0E4CFD9FF1200D9CFC7
:105D5000E5FFE1CFD9FF00C0E5FF01C0E5FF02C0CC
:105D6000E5FF03C0E5FF04C0E5FF05C0E5FF06C091
:105D7000E5FF020EDBCF00F0030EDBCF01F0040ED7
:105D8000DBCF02F0050EDBCF03F0046A056A0334B3
:105D9000066A063606B011D00250022603360350BA
:105DA000015C02E10250005C04E2D890033202324E
:105DB00004D0052A05C004F0EAD70350015C02E1D3
:105DC0000250005C04E30250005E0350015AD89078
:105DD0000332023204C005F004060550EEE101C0B2
:105DE000F3FF0050E4CF06F0E4CF05F0E4CF04F079
:105DF000E4CF03F0E4CF02F0E4CF01F0E4CF00F011
:105E0000E4CFD9FF1200E8CFE5FFD8CFE5FFE0CF20
:105E1000E5FFF3CFE5FFF4CFE5FFE9CFE5FFEACFFC
:105E2000E5FFFACFE5FFFBCFE5FFD9CFE5FFE1CFF7
:105E3000D9FF00C0E5FF01C0E5FFA1A23EEF2FF0B2
:105E400003012B51D8B431EF2FF09EEC24F0030165
:105E5000A26FD0C064F0D1C065F0D2C066F0D3C0EC
:105E600067F0A1920001D651006E016A0050B36E36
:105E70000001D551006E016A0050B26EE4CF01F00E
:105E8000E4CF00F0E4CFD9FFE4CFFBFFE4CFFAFF8B
:105E9000E4CFEAFFE4CFE9FFE4CFF4FFE4CFF3FF80
:105EA000E4CFE0FFE4CFD8FFE4CFE8FF10002563A4
:105EB00000000D0A0000080EF66E6B0EF76E000E65
:105EC000F86E0900F550056E0900F550066E04E104
:105ED000056702D0AAEF2FF00900F550006E090007
:105EE000F550016E0900F550026E09000900F550E9
:105EF000E96E0900F550EA6E090009000900F55045
:105F0000036E0900F550046E09000900F6CF07F092
:105F1000F7CF08F0F8CF09F000C0F6FF01C0F7FF97
:105F200002C0F8FF035002E1045009E00900F550F7
:105F3000EE6EF5CF7EFF0306F6E20406F7D707C044
:105F4000F6FF08C0F7FF09C0F8FF050601E20606E4
:105F500067EF2FF01200D9CFE5FFE1CFD9FF00C0E6
:105F6000E5FF01C0E5FF02C0E5FF03C0E5FF020E4B
:105F7000DBCF00F0030EDBCF01F0040EDBCF02F02D
:105F8000050EDBCF03F0005003019C6F01509D6FA5
:105F9000025003019E6F03509F6F03019C51030148
:105FA0009E03F3CF00F0F4CF01F000500301A06F87
:105FB0000150A16F03019C5103019F03F3CF00F037
:105FC00003019D5103019E03F3CF01F00150002610
:105FD0000301A15100260050A16FA1C3F3FFA051FE
:105FE000E4CF03F0E4CF02F0E4CF01F0E4CF00F01F
:105FF000E4CFD9FF1200D9CFE5FFE1CFD9FF00C030
:10600000E5FF01C0E5FF02C0E5FF03C0E5FF04C0F6
:10601000E5FF05C0E5FF020EDBCF00F0030EDBCF8E
:1060200001F0040EDBCF02F0050EDBCF03F00150D0
:10603000035C02E10050025CD8B027EF30F0025060
:10604000005C046E03500158056E2DEF30F00050D7
:10605000025C046E01500358056E05C0F3FF045046
:10606000E4CF05F0E4CF04F0E4CF03F0E4CF02F096
:10607000E4CF01F0E4CF00F0E4CFD9FF1200D9CF94
:10608000E5FFE1CFD9FF00C0E5FF01C0E5FF02C099
:10609000E5FF03C0E5FF04C0E5FF05C0E5FF006ABA
:1060A000016A080E015CD8B072EF30F0010E026E8A
:1060B000000E036E015006E0E86CD89002360336FD
:1060C000010FFCE327C304F0056A045002160550D3
:1060D000031602500310D8B46FEF30F0002A012AE3
:1060E00051EF30F00050E4CF05F0E4CF04F0E4CFFE
:1060F00003F0E4CF02F0E4CF01F0E4CF00F0E4CF0E
:10610000D9FF1200D9CFE5FFE1CFD9FF00C0E5FFED
:1061100001C0E5FF02C0E5FF03C0E5FF020EDBCFD3
:1061200000F0030EDBCF01F00050026E02500301BD
:106130002A6F0150E56E0050E56E020EE56E710E9D
:10614000E56EABEC2FF0006EF3CF01F0040EE1260C
:10615000026A036A00500008006E000E0156010E2C
:106160000256000E035600500001D56F0150000189
:10617000D66FE4CF03F0E4CF02F0E4CF01F0E4CF38
:1061800000F0E4CFD9FF1200D9CFE5FFE1CFD9FF6E
:1061900000C0E5FF01C0E5FF02C0E5FF03C0E5FF69
:1061A000020EDBCF00F0030EDBCF01F0040EDBCFDD
:1061B00002F0050EDBCF03F001C0E9FF02C0F3FFE0
:1061C000035013EC35F0A86E00C0A9FFA69EA69C54
:1061D000A684F29E550EA76EAA0EA76EA682A6A250
:1061E000F5EF30F00000EFEF30F0E86AA6B6E82AED
:1061F000A694F28EE4CF03F0E4CF02F0E4CF01F0F6
:10620000E4CF00F0E4CFD9FF1200D9CFE5FFE1CF12
:10621000D9FF00C0E5FF01C0E5FF02C0E5FF006E49
:10622000020EDBCF01F0030EDBCF02F0AC6AAB6AEB
:1062300000A001D0AC8800A202D0AC8CAB8C00A432
:1062400001D0AC8E00A602D0AB8801D0AB8A00A8EA
:1062500002D0AC8401D0AC949E9800AC02D09D8A50
:1062600001D09D9A9E9A00AE02D09D8801D09D9843
:106270000150AF6EAC8AAB8EE4CF02F0E4CF01F0F8
:10628000E4CF00F0E4CFD9FF1200D9CFE5FFE1CF92
:10629000D9FF00C0E5FF01C0E5FF02C0E5FF020E27
:1062A000D924006E000EDA20016E800E026E030EFD
:1062B0000026000E012202220250E56E0150E56E1A
:1062C0000050E56E040EDBCFE5FF030EDBCFE5FFEC
:1062D000020EDBCFE5FF0001FF51E56EFE51E56EDA
:1062E000FD51E56E69EC12F0006EF3CF01F0090E7E
:1062F000E12601C0F3FF0050E4CF02F0E4CF01F04B
:10630000E4CF00F0E4CFD9FF12000000000001004C
:10631000000000000000100000000000000000006D
:10632000000000000000000000000000000000006D
:106330000000000000000000000000080007000648
:10634000000500040003000200010000000000003E
:10635000000000000000000000000000000000003D
:10636000000000000000000000000000000000032A
:10637000000300A42400BA24000000000000000074
:106380000000D9CFE5FFE1CFD9FF00C0E5FF01C094
:10639000E5FF02C0E5FF03C0E5FF04C0E5FF020E14
:1063A000DBCF00F0016A026A080E015CD8B0ECEFA6
:1063B00031F0050E0224036E046A030E042203C0AA
:1063C000E9FF04C0EAFFFF0EEE6EFF0EEF6E022A39
:1063D000022A012AD4EF31F0005003012C6FE4CFE0
:1063E00004F0E4CF03F0E4CF02F0E4CF01F0E4CF17
:1063F00000F0E4CFD9FF1200D9CFE5FFE1CFD9FFFC
:1064000000C0E5FF01C0E5FF02C0E5FF03C0E5FFF6
:10641000020EDBCF00F0030EDBCF01F000C002F074
:1064200001C003F0FF0E0026D8A0010602500310A1
:10643000D8B429EF32F0010E026E036AFF0E022675
:10644000D8A0030602500310D8A41EEF32F00EEFBE
:1064500032F0E4CF03F0E4CF02F0E4CF01F0E4CF78
:1064600000F0E4CFD9FF1200D9CFE5FFE1CFD9FF8B
:1064700000C0E5FF01C0E5FF02C0E5FF03C0E5FF86
:10648000020EDBCF00F0030EDBCF01F0040EDBCFFA
:1064900002F0050EDBCF03F00150035C02E1005077
:1064A000025CD8B056EF32F05AEF32F002C000F082
:1064B00003C001F001C0F3FF0050E4CF03F0E4CFCC
:1064C00002F0E4CF01F0E4CF00F0E4CFD9FF1200F6
:1064D000D9CFE5FFE1CFD9FF00C0E5FF020EDBCF4A
:1064E00000F0110E005CD8B07AEF32F00050D8A462
:1064F0007DEF32F0E86A84EF32F000500301296F3B
:1065000000C06CF003012951E4CF00F0E4CFD9FFC3
:106510001200416374697665206368616E6E656C14
:10652000733A20005B25642028256C64295D2000D7
:106530000D0A0000D9CFE5FFE1CFD9FF00C0E5FF8C
:1065400001C0E5FF02C0E5FF020EDBCF00F0005006
:10655000200DF3CF00F0F4CF01F0000E0026010E65
:1065600001220150016E0050006E800E026E02C0CA
:10657000F4FF01C0F3FF0050E4CF02F0E4CF01F0DC
:10658000E4CF00F0E4CFD9FF1200D9CFE5FFE1CF8F
:10659000D9FF00C0E5FF01C0E5FF02C0E5FF020E24
:1065A000DBCFA9FF030EDBCF00F0040EDBCF01F041
:1065B000050EDBCF02F0A69CA69EA680A8CFE5FF25
:1065C00000C0E9FF01C0F3FF02504EEC35F0E4CF0C
:1065D00002F0E4CF01F0E4CF00F0E4CFD9FF1200E5
:1065E000D9CFE5FFE1CFD9FF6D966F86D00E926EC1
:1065F000806A0F0EC16E936A816AA10E946E826AE0
:10660000000EE56E0A0EE56E7C0E05EC31F0020E12
:10661000E1260001FD6B0001FE6B200E0001FF6F03
:106620000301996B03019A6B200E03019B6FE4CF6A
:10663000D9FF1200D9CFE5FFE1CFD9FF00C0E5FFB8
:1066400001C0E5FF020EDBCF00F00050030104158E
:10665000016E0150D8B430EF33F0020E3BEF33F04F
:106660000301035100160050D8B43AEF33F0010E85
:106670003BEF33F0E86AE4CF01F0E4CF00F0E4CF81
:10668000D9FF1200D9CFE5FFE1CFD9FF00C0E5FF68
:1066900001C0E5FF020EDBCF00F0010E016E0050DD
:1066A00005E0E86CD8900136010FFDE3011C006E97
:1066B00003012751001600500301276FE4CF01F0BA
:1066C000E4CF00F0E4CFD9FF1200D9CFE5FFE1CF4E
:1066D000D9FF00C0E5FF01C0E5FF020EDBCF00F0EF
:1066E000010E016E005005E0E86CD8900136010FF4
:1066F000FDE3015003012711006E00500301276FD5
:10670000E4CF01F0E4CF00F0E4CFD9FF1200E8AE0F
:106710000AD0F3CFEAFFEE50EECFF3FFEECFF4FF57
:10672000EECFE9FF1200E8BC11D0E9CFF6FFF3CFBE
:10673000F7FFF86E0900F5500900F5CFF3FF0900E7
:10674000F5CFF4FF0900F5CFE9FF12001200D9CF11
:10675000E5FFE1CFD9FF00C0E5FF01C0E5FF020E74
:10676000DBCF00F0001C016E030104510116015043
:106770000301046F0050E56E90EC1CF0E12AE4CFB9
:1067800001F0E4CF00F0E4CFD9FF1200D9CFE5FF4C
:10679000E1CFD9FF00C0E5FF01C0E5FF020EDBCF6E
:1067A00000F0001C016E03010351011601500301AA
:1067B000036F0050E56E90EC1CF0E12AE4CF01F08D
:1067C000E4CF00F0E4CFD9FF1200D9CFE5FFE1CF4D
:1067D000D9FFCC6ACA6A7D0ECB6E500ECA12CA802F
:1067E0000001D06B0001D16B0001D26B0001D36BB3
:1067F000CA84B36AB26AB18EB192B18AB188B180EB
:10680000E4CFD9FF1200D9CFE5FFE1CFD9FF00C017
:10681000E5FF01C0E5FF020EDBCF00F000500301F1
:106820000319016E01500301036F0050E56E90ECF7
:106830001CF0E12AE4CF01F0E4CF00F0E4CFD9FF6F
:106840001200D9CFE5FFE1CFD9FF00C0E5FF01C0BD
:10685000E5FF020EDBCF00F0005003010311016ED3
:1068600001500301036F0050E56E90EC1CF0E12A2B
:10687000E4CF01F0E4CF00F0E4CFD9FF1200D9CF8C
:10688000E5FFE1CFD9FF00016D2BD8A002D00001B8
:106890006E2B000E00016E5D03E1330E00016D5D95
:1068A000D8A059EF34F038EC23F000016D6B0001F3
:1068B0006E6BE4CFD9FF1200E8AE08D0F3CFEAFF49
:1068C000EE50EECFF3FFEECFF4FF1200E8BC0ED097
:1068D000E9CFF6FFF3CFF7FFF86E0900F550090096
:1068E000F5CFF3FF0900F5CFF4FF12001200D9CF66
:1068F000E5FFE1CFD9FF00C0E5FF020EDBCF00F0DE
:10690000610E005C05E37B0E005C02E2010E01D02B
:10691000E86AE4CF00F0E4CFD9FF1200E8AE06D079
:10692000F3CFEAFFEE50EECFF3FF1200E8BC0BD03E
:10693000E9CFF6FFF3CFF7FFF86E0900F550090035
:10694000F5CFF3FF12001200D9CFE5FFE1CFD9FF59
:10695000D59ED59CD58AD586CD90CD8ECD9CCD9615
:10696000CD82CD9ACD98D58ECD80E4CFD9FF1200BF
:10697000D9CFE5FFE1CFD9FF00C0E5FF020EDBCFA5
:1069800000F003010451001200500301046FE4CF32
:1069900000F0E4CFD9FF1200F00E0301A615A66F98
:1069A000ABAC04D0A691ABA001D0A681ABA402D021
:1069B0000301A685ABA202D00301A687AE50120048
:1069C000D9CFE5FFE1CFD9FF00C0E5FF020EDBCF55
:1069D00000F000500301276FE4CF00F0E4CFD9FFAF
:1069E0001200D9CFE5FFE1CFD9FF8080000EE56E20
:1069F000010EE56E98EC29F0020EE1268090E4CFBE
:106A0000D9FF1200D9CFE5FFE1CFD9FF00C0E5FFE4
:106A1000020EDBCF00F000500301286FE4CF00F03E
:106A2000E4CFD9FF1200E8AE04D0F3CFEAFFEE5076
:106A30001200E8BC08D0E9CFF6FFF3CFF7FFF86EFD
:106A40000900F55012001200D9CFE5FFE1CFD9FFC0
:106A5000D08EF28EF28C9D829F92A082A2829D8A1D
:106A60009F9AE4CFD9FF1200E8AE09D0F3CFEAFF36
:106A7000E4CFEEFFF4CFEEFFF6CFEEFF1200E8AC6E
:106A80001200120012EEFFF022EEFFF0F86AA68E5E
:106A9000A69C5BEC2FF05AEC1FF0FFD7E8AE05D0B8
:106AA000F3CFEAFFE4CFEEFF1200E8AC12001200D1
:106AB000D9CFE5FFE1CFD9FF03012A51E4CFD9FFB8
:106AC0001200D9CFE5FFE1CFD9FF03012751E4CF71
:106AD000D9FF1200D9CFE5FFE1CFD9FF00016C51FA
:106AE000E4CFD9FF1200D9CFE5FFE1CFD9FF0301F1
:106AF0002851E4CFD9FF1200D9CFE5FFE1CFD9FF6C
:106B00001200E4CFD9FF120001000A630000600008
:106B1000000078000000ACA2FED7AD6E1200E8CFF6
:086B20007FFF1200C96E120094
:020000040030CA
:0E000000C43CF8E0FFFC9AFFFFFFFE9FFFFFED
:00000001FF
